:020000041100E9
:103000007FB50023284C294D03932800217C284AB2
:1030100001F0E5FA002812D103232800217C03AA3D
:1030200001F084FA00280AD1224B039A9A4206D171
:10303000214B2248E360224B636104B070BD02263D
:10304000217CFE2228001F4B009601F041FA002847
:1030500001D00020F1E71C4BA2899A42F9D1217CD2
:10306000FF222800194B009601F032FA0028F0D117
:10307000E389174A934203D1164B17486361DCE793
:10308000164A9342E5D1164B164A1B68934206D95D
:10309000C02304222800217C9B0001F082FA124BFD
:1030A00012486361C9E7C046F461FF1F3442FF1F45
:1030B000813700005959530059598320E4BA00114F
:1030C000114200110062FF1F595900000262FF1FE8
:1030D00083050000C5410011C4BA0011821500002B
:1030E0001862FF1F87130000CD420011D4BA0011EF
:1030F000002370B51A4E1B4C30006361637401F0FD
:1031000095F9402323744B2B0CD9CC233821AC22C6
:1031100030009B01217401F044FA00280AD00025F8
:1031200025740CE0FFF76CFF051E08D1237C0433E7
:10313000DBB2E7E70C4B0D4D63610D4BE381236878
:10314000002B08D1002D06D00C222900200008F009
:1031500003FC2B7B6374300001F0A6F970BDC04600
:103160003442FF1FF461FF1F65420011B4BA001121
:10317000AAAAFFFFF7B5164B0192C318021D002043
:10318000009388235B05D3181B685C1C1AD09CB283
:10319000402C18D88D781E0CAC466746CD782D0291
:1031A0003D43AE4206D1019800280ED110000C70AC
:1031B000240A4C7003249BB20733A343D218009B0C
:1031C0009A42DED3FEBD4432F9E71000FAE7C0466A
:1031D000FC0F0000802213B503000324019189B283
:1031E000520107319B18A14304305A1A88235B050A
:1031F000C3181B68591C03D190429241104016BD60
:1032000099B2402907D80B000733A343C018904256
:10321000ECD30020F3E74430F9E7134B134A1B6863
:10322000126810B5FA24934201D81A00F824104B02
:10323000E4021B689A4210D813000E4A12689A42A0
:103240000ED3013307D1F823DB029C4203D10A4994
:10325000054808F0B1FB200010BDFC24E402ECE7B7
:10326000FE24E402F7E7C04600C0071100D00711B2
:1032700000E0071100F00711FFFFFF7FF0B59BB0E2
:10328000150004900391402A00D9A0E006AB5980B4
:103290001A80FFF7C2FF0400042816D9002206A9ED
:1032A000FFF768FF052810D906AB1B88AB420CD18D
:1032B000002D07D0514B2A000499C01808F0DCF803
:1032C000002802D101201BB0F0BD06AB1D802000FC
:1032D0000699FFF77FFF041E7BD1069B0793FFF73C
:1032E0009CFF80235B01C618802307001B039E42BE
:1032F00001D3F826F60288235B05F31801931B68B7
:10330000013302D0019808F04FFA3D49019808F0C6
:1033100053FB3B1D0293331D05938822029B5205EC
:103320009B181B6808935A1C3CD044219AB2009108
:10333000402A04D80320D11D814389B2009103990A
:103340001B0C8B4224D0402A22D80122300008A92D
:10335000FFF710FF021E1BD1380008A9FFF70AFF74
:103360000400042831D9009A059B9B188022520141
:10337000B218934240D288235B05C118009A09A86D
:1033800008F0EAFA1D4B009A09A9F01808F024F891
:10339000009A029B9446634402931A4B029AFB18CC
:1033A0009A42BAD388235B05FC1821680198013939
:1033B00008F002FB200008F0F7F9039A07AB5A80E7
:1033C00030000799FFF706FF0400002C03D100200E
:1033D00079E70428FBD988235B05E018069908F0F3
:1033E000EBFA0323EA1C9A4300D16BE7034B0499E1
:1033F000E01807F0F1FF65E70424ECE70400001192
:10340000FFFFFF7FF80F0000F7B505001400402A0A
:1034100021D8002701AE71803780FFF7FEFE042817
:1034200016D93A003100FFF7A5FE042810D93688D6
:10343000BC420BD0BD4209D0221CB44200D9321C80
:10344000064B92B2C118280008F086FA30B2FEBDD1
:10345000C04300B2FBE703204042F8E7040000113C
:1034600037B5042204000D0001A81649FFF7CCFF70
:10347000020004280BD1019BA34208D3AB4204D025
:10348000104901A80195FFF7F9FE01203EBD0E4C41
:1034900023682000019308F087F901992000013981
:1034A000019108F089FA80235B01E418074B9C42E4
:1034B000EED10422034901A80195FFF7DFFE0020A9
:1034C000E4E7C0465555000000C007110000081190
:1034D00030B589B008F030F810226946254808F068
:1034E0006BF9254B009A9A420ED1019B029A0F2B41
:1034F00033D8002101240698013B08D2002900D0CE
:103500000292029B013331D10023029325E0551C26
:10351000F2D102002100EFE710341022200004A9AC
:1035200008F04AF9029B013301D1069B02938823DC
:1035300004995B05C918059B06981A03120B0491A0
:103540000592814203D02B4201D108F005FA019B7C
:10355000013B0193019B002BDED1029B002B03D08A
:10356000049304984168084709B030BDE025014C38
:103570002D03EFE700000111504859368022F8B5BD
:10358000964C974BD200002120001C6007F0FCFEF7
:103590002300944A88331A60934B1A786A23002ACE
:1035A00000D01133E3620A232365904B37221B7846
:1035B0000820A3638E4B2118E361102323628D4BF7
:1035C0003B256361C823DB00A36123008C331A60B1
:1035D0002823013AE26320646364CA67043A211D28
:1035E000CA672100BC310D602100C0310860210094
:1035F000C4310B6021000635CC310D602100083D3F
:10360000C8310D602100D0310A602200D432106030
:103610002200D832136022000227E0322100176016
:103620004222DC310A6021001B3DE4310D602100A3
:10363000E83108602100EC310B6023000521F433F0
:1036400019602300F0331A602300183290331A6097
:1036500023009433186023001E3A98331A60AF2376
:10366000DB002360644BFA262363644B644DE36004
:10367000644BF031A3642300FF31FC33B600A1603A
:1036800021611E60A5627325E5656D3D6565A565D3
:1036900096255D4AAD00E264666258606766A5667D
:1036A00000270925A767E566584F594D6067200038
:1036B0002567E2673A6015279C30676007001A208B
:1036C00038602000A0300700212038602000A8309A
:1036D00007004C4838602000F83006602600642758
:1036E000A436376026005F3FAC3637602600033FC4
:1036F000B03637602600C637B4363760260000275C
:10370000B836376038269E60424E96205E64424E40
:103710005A66DE61414E9A645E62F53EFF3E9E62ED
:103720001E269A67354A8000DE661F675F67DD6583
:103730001D661862DA67BE23394A5B00E250394BD6
:10374000D838235004302250C4225200A350C6233C
:10375000E4205B00E1500433334AE1503349344BF9
:10376000D1603449800019503349E938FF38195085
:1037700032490430195032493248D161324911631B
:10378000324951631900F4310860CE2030494000BD
:1037900011603049195019002F48F83108602F493D
:1037A000D16582212E4A89005A501A002D490832CB
:1037B000D1671A002C49B432116088212B4A890044
:1037C0005A501A002A49883211602A4ADA6408F0ED
:1037D000DBF8012007F020FEF8BDC0460004FF1F03
:1037E0009064FF1F606FFF1F6444FF1F4A0AFF1FA2
:1037F0003A07000080C3C9019A020000DC050000FE
:103800006A18000050C3000088130000F009FF1F71
:10381000204E00006509FF1F68100000C409000069
:1038200040420F0010270000FC00FF1FB11CFF1FCB
:103830000000FF1F052DFF1F8D30FF1F252FFF1FCD
:103840007120FF1F6127FF1F8D20FF1F3922FF1FDF
:10385000FD1FFF1F8529FF1F6D2AFF1F8D19FF1FE9
:103860009128FF1FB525FF1FC125FF1FFD1EFF1F4C
:10387000B51FFF1F751EFF1F0223F0B50124644D05
:10388000644E2B70644B91B01C70644F039333688B
:10389000002108207B7006F071FC082006F068FB10
:1038A0000023984205D07A78552A02D0332A00D0D6
:1038B000A1E03360042006F0DBFD07F0F5FDFFF723
:1038C0005DFE08F029F81F2201240021544B10AEA0
:1038D0001A70544B1C70544B1970544B1968914317
:1038E000163A0A431A60602219689143403A0A4323
:1038F0001A6007F0D1FF07F02FFE4D4B9847C1200B
:10390000FF214C4B80001A588A431A50C52292005E
:1039100098588843BF390143995098584649084000
:103920008021C9010143802099509958C00509029E
:10393000090A0143995080214048490107F0E4FEFB
:10394000032322003E49019400933E4807F0DCFD2A
:103950002C223D4905A807F0FFFF05AC61782078CF
:10396000023406F025FBA642F8D1384C0121002094
:1039700006F032FC0920012106F02EFC2268344BAF
:1039800003201A40A023DB02134323608023226814
:103990009B041343236022682E4B1A4080239B0311
:1039A000134323602C4A2D4B934200D8012007F08B
:1039B00073FD07F0A9FF80232268DB041343236013
:1039C000287807F0E9FF039B1878C0B207F064FE7F
:1039D00007F032FD2249042007F0EEFD06F014FD49
:1039E00000F040F800F014FE00F0BCFE00F018FA01
:1039F000002011B0F0BD00932100194A042007F007
:103A00006BFE8023DB059C62FFF762FD52E7C04638
:103A10004A0AFF1F34F000406444FF1F2462FF1F66
:103A2000480AFF1F490AFF1F680AFF1FBCF0004039
:103A3000E1A2000000E100E0FF00FFFF6844FF1F7B
:103A4000EC56FF1F6854FF1FD8B9001114F0004056
:103A5000FF7FF8FFFFFF9FFF0080FF1F606FFF1FCA
:103A60003B000108002210B51100112007F0ACFC4A
:103A700010BD0000F8B500230926374F374C3B62D4
:103A8000E3681120B343E36007F096FC112007F0D0
:103A90006BFF112007F0E0FD4023226880251343CF
:103AA000236080236268DB0213436360A3682C4AAF
:103AB0002B43A360A36802211340A3608023A26864
:103AC0009B0113431022A360236C072093432364BC
:103AD000236C0F3A1343236480235B003B62226B09
:103AE000204B1A402263626B1A406263A26B1A4039
:103AF000A263E26B1340E363E3681B4A1340E36095
:103B000006F056FA0121072006F066FB174B11203C
:103B10005A6C15435D6407F01FFEFD21144B154AD6
:103B200089005A508023C720626B5B031343636391
:103B3000E36880003343E3600F4B104A195811408B
:103B4000802212020A431A50802292051A6008222B
:103B50000B4B5A63F8BDC04600F000403CF00040FB
:103B6000FFFFDFFFEFFFEFFFFFFF7FFF00380040A9
:103B70000000FF1F5118FF1F00E100E0FF00FFFFE2
:103B800000000540E12010B5C00407F0CDFD10BDD8
:103B900070B52B4C238C002B2AD0FA22D2009342F2
:103BA00001D2FFF7EFFF228A238C002A21D1DA000D
:103BB00023826382A382E38223836383A383E383D9
:103BC00022606260A260E2601E4D1F4A6420EB80AA
:103BD00093420AD8FA220020D200934205D91B4A08
:103BE0000A21981807F010FDC0B200232872238420
:103BF00070BD0720E11CCA7F01320240CA7705D19F
:103C00000325201DC17F01312940C17708325200B0
:103C1000A352002321001A00088A01321B18023126
:103C2000082AF9D1221DD27F9200A350626823682E
:103C30009B18A2689B18E2689B185B099BB2C3E7BC
:103C40006461FF1F0C62FF1FB70B000030F8FFFF1D
:103C500030B503A804880B20002C0ED14968074D0D
:103C600008784978090201430A20A94205D10121B7
:103C700020001980024B1B7A137030BD192A0000F6
:103C80000C62FF1FF7B5150008AA16884A680F4F87
:103C900014785278120222430A24BA4214D1012223
:103CA000DBB2019200962A0007F0FEFA041E0BD147
:103CB000074B1B68002B07D068782A780002104356
:103CC00042425041013098472000FEBD02290000C9
:103CD0009061FF1F30B5012503790400BFB02B426E
:103CE00011D00A49408806F04BFE28420BD0084B01
:103CF00001A95B8D4D800B80064B00221B7A6088EA
:103D00000B7103F01DFF3FB030BDC0468861FF1F3F
:103D1000A840FF1F0C62FF1F10B50549054806F0BB
:103D2000E5FD0421044A054806F0A2FD10BDC04689
:103D30008861FF1FFFFF000004BA0011A840FF1FA9
:103D400010B5024804F07EFD10BDC046D53C001100
:103D5000012303700B4B1A7A4270022282709A7808
:103D6000C270DA780271032242711A7982715A792B
:103D7000C2710C2202729A794272DB7983720B2033
:103D80007047C0460C62FF1F022310B50370013B51
:103D900043700533837010330371443B43712A33FE
:103DA00083714433C37100230372064B04001B88E4
:103DB00043720A30FFF7CCFF831D0A30C0B2E370B4
:103DC00010BDC0460C62FF1F10B5142007F04CFC5C
:103DD000124B14220021186007F0D6FA002007F0D9
:103DE000B3FD012007F0D0FB022007F0DDFB03202C
:103DF00003F0CCFF042005F0E1FF052003F00AFAF0
:103E0000062003F0D7FE072001F06EFA082006F026
:103E10000FFD092001F040F810BDC0469461FF1F5E
:103E200007F0C2FD012007F08FFC07F09DFB0000AA
:103E3000094B10B50400984205D0012904D1200097
:103E4000064906F053FD10BD0229FCD1013904F0EA
:103E5000B7FC0028F3D0F6E7FEFF0000BA61FF1FB1
:103E600070B50D7A100004AA2C0016881022144098
:103E7000154220D1002E20D10A78022A18D14A6892
:103E8000517815780E4A09022943914205D00D4A0E
:103E9000914209D01C800A2404E014220A491A80A5
:103EA00007F05AFD200070BD0C2208491A80F7E780
:103EB0001C800124F6E70824F4E70B24F2E7C0464F
:103EC000F3FF0000F4FF0000F042FF1F00BB0011F1
:103ED00010B504000749084806F008FD074804F03B
:103EE000F1FB0020E40704D50721054A054806F048
:103EF000BFFC10BDBA61FF1FFFFF0000313E001183
:103F000048BA0011EC40FF1F00B50C4BBFB01A7847
:103F10000B4902A800F0E0FC6B4680B2D880002874
:103F200009D06A46074B01A91B889380064B0022E3
:103F3000188803F005FE3FB000BDC0469861FF1F22
:103F40009961FF1F4641FF1F5042FF1F00B50C4BF8
:103F5000BFB01A780B4902A801F038FD6B4680B259
:103F6000D880002809D06A46074B01A95B8D938051
:103F7000064B0022188803F0E3FD3FB000BDC046A9
:103F8000C261FF1FC361FF1FEC40FF1F5042FF1FB4
:103F9000F7B50E00377A1C0008AB11003D001A88F7
:103FA00020231D401F423CD13378022B3BD1736844
:103FB0001F785B781B023B431E4FBB4208D01E4F4D
:103FC000BB4214D01D4DAB4221D00A252800FEBDB6
:103FD000002A2AD1142C2AD82200F06807F0BCFC51
:103FE000174B1C70012CF1D9FFF7B0FFEEE7002A48
:103FF0001BD1202C1BD82200F06807F0ADFC114B20
:1040000004211C70104B187807F03EFADEE7E3B28B
:104010000124009201940A00310007F045F90500DF
:10402000D4E70825D2E70125D0E70B25CEE70D25FB
:10403000CCE7C046F3FF0000F4FF000002290000B7
:10404000C261FF1F9861FF1F4462FF1F332310B539
:10405000040003700A220749013007F07DFC064B7B
:104060000F201B681A0AE37222731A0C1B0E62736C
:10407000A37310BD0C62FF1F3462FF1F30B5012512
:1040800003790400BFB02B4213D00B49408806F0DF
:1040900077FC28420DD06A46084B02A81B88938003
:1040A000FFF7D4FF6B46D8800022608801A903F097
:1040B00047FD3FB030BDC046BA61FF1F4641FF1FFC
:1040C00010B5024804F0BEFB10BDC0467D40001193
:1040D00070B5160004AA148805AA15784A685078A5
:1040E000117800022A4A0843801805284BD807F0A7
:1040F0007BFB03131E29343F0720042C0BD8052219
:10410000121BAA4200D92A0022491A80300009193C
:1041100007F022FC002070BD0720112CFBD81222D2
:10412000121BAA4200D92A001B491A80EEE7072079
:104130000E2CF0D80F22121BAA4200D92A001749D0
:104140001A80E3E70720032CE5D80422121BAA42B9
:1041500000D92A0012491A80D8E70720032CDAD8A0
:104160000422121BAA4200D92A000E491A80CDE768
:104170000720032CCFD80422121BAA4200D92A0000
:1041800009491A80C2E700220A201A80C3E7C04604
:10419000DCD5FFFF93BA0011E061FF1F83BA001165
:1041A0007EBA001179BA001174BA001110B50D2150
:1041B000024A034806F05CFB10BDC04668BA001115
:1041C0005C41FF1F13B5104C0423217C01AA00F0B1
:1041D000ADF9002815D16B469A88236852BA92B27D
:1041E0005343228909491B0C9B184B806B46DA8884
:1041F000636852BA92B2534362891B0C9B188B803E
:1042000016BD0120FCE7C046F461FF1F0C62FF1FD2
:1042100013B5124C06236A46217C00F087F900286A
:1042200019D16B461988236849BA89B24B43218951
:104230000B4A1B0C5B1853806B46D97803335B78B1
:104240001B020B435BBA61689BB24B4361891B0C39
:104250005B18938016BD0120FCE7C046F461FF1F88
:104260000C62FF1F37B5174C07236A46217C00F00C
:104270005DF9002824D16B461B787F2B20D86B4634
:10428000DD78F0232A041B031A406B469B880E49F5
:104290005BBA9BB21A4323682D09534322891B0C36
:1042A0009B184B806B465A789B7812031B011A436C
:1042B00063682A43534362891B0C9B188B803EBD65
:1042C0000120FCE7F461FF1F0C62FF1F7FB502268F
:1042D000154C0022217C03AB0096050000F0F8F895
:1042E000002802D0012004B070BD0E23217C0122E1
:1042F000280000966B4400F0EBF80028F2D16B46E2
:104300009A892368D2BA5343228908491B149B18FF
:104310004B806B46DA89636852BA92B25343628922
:104320001B0C9B188B80DEE7F461FF1F0C62FF1FE4
:1043300070B5184C237C002B0FD0382B0ED1164DA6
:10434000280000F073F8CC23AC222800217C9B01CC
:1043500000F027F9280000F0A7F870BDE3890F4AA4
:10436000934209D10C4D280000F060F8002228008B
:10437000217C00F005F9EDE7094A9342EDD1064DA5
:10438000280000F053F890222800217C920100F0D0
:1043900026F9DFE7F461FF1F3442FF1F83050000A9
:1043A0008320000070B5144C237C002B1FD0636960
:1043B000002B1CD0114D280000F038F8636928004C
:1043C00098470400280000F06FF8002C10D10C4B27
:1043D0000422995E002905DA9C801A8801321A802D
:1043E000200070BD074A9142F7DD9A80F5E701246D
:1043F000FEF77EFEF4E7C046F461FF1F3442FF1F64
:104400000C62FF1F0F27000010B58024064AA4008D
:104410001168436B234205D113685B1A032BF8D94B
:10442000012010BD0020FCE76008FF1F70B5C179B6
:1044300005000C00631E9C411A4BE402E41849007D
:104440000460C9B2007905F0FDFEE9796879490098
:104450000131C9B205F0F6FEE8790930C0B207F0C3
:10446000FBF80023E36661332360AA795B3B002AF3
:104470000ED022689A43023B134323600A23E36170
:104480000733236200232363A3630133E36370BD17
:1044900022689A4302231343236046236361063351
:1044A000A361EFE70050004070B5002504000368E9
:1044B000DD66C0790930C0B206F07EFF29002079A0
:1044C00005F05CFE2900607905F058FE70BD000023
:1044D000F8B51E0006AB1D78002304681700E366DC
:1044E000616007F029F801238022E3662B00276131
:1044F0005200013B08D207F09FF908200A4A1168D0
:10450000002D03D12800F8BD2261F2E7236F03429A
:1045100003D02369013D3370013613685B1A032B06
:10452000EED90125EEE7C0466008FF1F70B51C00FC
:10453000002305681600EB66696006F0FDFF0123A5
:104540008022EB6623005200013B08D207F074F989
:1045500008200A4A1168002C03D1200070BD2A618E
:10456000F2E72B6F034203D02B69013C3370013615
:1045700013685B1A032BEED90124EEE76008FF1FD6
:10458000002370B504681500E366616006F0D4FF8F
:104590000123E366256107F04FF92000FFF734FFA0
:1045A00070BD70B51D00002304681600E3666160ED
:1045B00006F0C2FF0123E36626610F33626B1A42E5
:1045C000FCD02B0A23611023626B1A42FCD0EDB29F
:1045D000256107F031F92000FFF716FF70BD0023B9
:1045E00070B504681500E366616006F0A5FF01235D
:1045F000E3662B0A23611023626B1A42FCD0EDB2F2
:10460000256107F019F92000FFF7FEFE70BD0000DC
:1046100010B5084CE368002B08D18022064B5202EB
:104620001B689B186360054B1B68236007F02CF91F
:10463000A06010BD3462FF1FC8F00040CCF0004005
:1046400070B5184A936A916A9942FBD116498A68F3
:104650009A421FD39A1A8B60144B0126186893B2A2
:10466000D202D20E4343424300204C681B0A1B195E
:1046700012029B180E4C0A684B60551CA3420CD8C2
:10468000002801D04B600A600A4A136008680A4B90
:10469000186070BD581E821ADDE7084A30009B186A
:1046A0002A00EAE700F000403462FF1F140AFF1FEF
:1046B00040420F00C8F00040CCF00040C0BDF0FF09
:1046C00070B51F4C23793F2B01D93F2323711D4B1C
:1046D00022791A701878C0B206F01EFF18231A4902
:1046E0001A4A0B801A4913800B805380A379194909
:1046F00080200B800C21938001334B43164D191CF5
:104700000001834200D9011C2980D1806379002BEC
:1047100001D101336371237A012B01D80223237263
:104720006279237A0D4853430A21584306F06CFFFF
:104730000B4D2860E379052B01D81023E37170BD80
:104740002862FF1F480AFF1F4E42FF1F1044FF1F31
:104750004C42FF1F4A42FF1F4842FF1F71020000E8
:104760001862FF1FF8B520210020FEF779FE114CDA
:10477000011E114D09D10C22104BC1CBC1C4280020
:1047800006F002FEFFF79CFFF8BD0C2220000C494A
:10479000FEF73AFE0C2802D0084B43CB43C40C2250
:1047A00028000849FEF730FE0C28EBD00C2200212F
:1047B000E5E7C0462862FF1FF461FF1FF4BA00114D
:1047C000FC0C0000F50C0000F0B51D4C8022A54447
:1047D0000400882069465201400506F025FF90221A
:1047E00012016A441300200032C832C316C816C32F
:1047F0008023144C144FA6689B033343A3603B6093
:1048000006F0CAFE8823A0685B05C01806F0CCFF3E
:104810000025882329008022A0685B05C018401964
:104820006944520006F0D8FD80230135FF355B0155
:104830009D42EED1A6603E60044B9D44F0BDC04653
:10484000FCEFFFFF8043FF1F9808FF1F04100000CC
:10485000F0B5040087B0002825D0684606F0C4FDF6
:104860001B4C022806D106226946200006F004FEF1
:10487000002816D06946002301250F262F00E25C90
:10488000013310091030874038002F003240974024
:104890003A0002434A610439062BEFD16846FFF71C
:1048A00093FF07B0F0BD182269460A4806F0BCFE27
:1048B0006A46A300D358013305D01822FF21684669
:1048C00006F062FDEAE70134062CF1D1E9E7C046C3
:1048D0006509FF1F00090011F0B5002504000E0056
:1048E00085B0AA4200D183E04B1C087801934B7835
:1048F0008978377909021943F3783F061B040B4383
:104900001F43039720706570252800D193E033D8AA
:10491000112813D806F040FD660017011701170192
:104920001701A700B500AE00170117011701170105
:104930001701170117011701F1001101232800D1F8
:10494000CAE0DB2800D020E1042A00D8AEE0102520
:10495000052A05D0551F2A003800711D06F0FCFFFE
:1049600005223100200006F0F7FF2A003900601D03
:1049700006F0F2FF05353BE0562856D010D8332814
:1049800000D1A4E0552836D02628DAD18E4B290054
:10499000132218001D0006F0F7FCFEF7A9FB59E0F2
:1049A000712800D174E0722800D186E0DC28C8D1DB
:1049B000022A00D87AE07378BFB26370B378A3702C
:1049C000032A05D0033A390092B2F01CFEF756FCD8
:1049D00010223900E01CFEF717FDC51C002807DA7D
:1049E000607070E00C222000784906F0B5FF0C25BD
:1049F000280005B0F0BD013A754D0C2A13D8002AE5
:104A00000AD02800019906F0A7FFFFF759FE0C22F3
:104A100028007049FEF732FC29000C22601C06F0C9
:104A20009BFF0D25E4E70C22EBE7694D6A4B2A005A
:104A300043CB43C2E9E7013A634D0C2A11D8002A5F
:104A400008D00199280006F087FF0C22280063494E
:104A5000FEF714FC29001322601C06F07DFF1425CC
:104A6000C6E70C22EDE706225D49601C06F074FFE4
:104A70000625BDE712225B49601C06F06DFF132579
:104A8000B6E708225849601C06F066FF0925AFE723
:104A9000012A0ED07178F02908D8544D288801F0E9
:104AA000F1FB534B2A885200D35A00E0FF23637076
:104AB00009E04E4A4E4B1288F5E74E4B012A04D0CE
:104AC00072781A706270022592E71B78EFE7200077
:104AD000FFF7BCFA05008BE7042A04D9464D2F6086
:104AE00006F0D2FEA860FFF7ABFD0422039003A9F5
:104AF000601C06F031FF05257AE7404D062A15D9DE
:104B000006222800019906F0B7FC00280ED00622E4
:104B10000199280006F020FF062239492800FEF7F7
:104B2000ADFB0123334A11780B4313702900062291
:104B3000601C06F011FF07255AE7012AB6D07078ED
:104B4000FFF786FEBFE7012800D0FAE6931E2D4F3F
:104B5000132B06D87378002B0BD100F00BF900F063
:104B600041F9294B39001D78601C6A1E06F0F4FEDD
:104B70003EE7551E2A000199380006F0EDFE380088
:104B80002249AAB2FEF77AFBE9E7DA288ED1042A95
:104B90008CD9082A15D9B37972791B021343F2799B
:104BA00012041A43337A1B0613433B603B68052209
:104BB00031002000039306F0CFFE0422601D03A9FC
:104BC00062E7FE236370F1E7F461FF1F00BB001191
:104BD0002862FF1FFC0C0000F4BA0011F50C000065
:104BE0000062FF1FE061FF1F8443FF1F5042FF1F51
:104BF0009464FF1F2462FF1F3462FF1F6509FF1FBB
:104C0000ADAC00002564FF1F2364FF1FAEDE000073
:104C100070470000020010B5094B0A32094C92B2ED
:104C2000DA815A8298811882207802F091F9042260
:104C3000054B012120781A7006F026FC10BDC046F5
:104C40000E43FF1F6E64FF1F6D64FF1F013870B5B8
:104C5000042809D806F0C8FD0309230812001E4BDA
:104C60000221187806F010FC70BD1B4B0821187843
:104C700006F0DAFB0022194B1A72F5E780220024B5
:104C8000164B154D52001A81082128781A68DC72DB
:104C900006F0FAFC2100287806F0AEFDE4E70E4BA2
:104CA0000821187806F0C0FB0D48FFF76DF80D4B92
:104CB0000D4A9B7993800D4A13800022074BDA72CC
:104CC0000132FF321A810A4B1B78002BCCD0094AE3
:104CD000136006F079FDC7E74462FF1F1862FF1FEB
:104CE0005942FF1F2862FF1F1044FF1F4A42FF1F47
:104CF0002462FF1F34F0004010B500290FD10828AE
:104D00000DD10131013005F067FA054B1B78002BFE
:104D100005D02622034B04485A72FFF77BFF10BDD3
:104D20004664FF1F1862FF1FC409000010B5012967
:104D300005D1082803D10021013005F04DFA10BD3E
:104D40000300F0B50A4D8E18B14202D1520080180E
:104D5000F0BD0C782F6824093C5D0F271C700C787F
:104D600001313C402F683C5D5C700233ECE7C0468B
:104D70004442FF1F0E22124B10B51A700D23114C26
:104D800011492370093A043B1048637006F0E4FDB2
:104D90002D2301220E490F48E371FFF7D1FF0122B5
:104DA0000D49FFF7CDFF01220C49FFF7C9FF0300B2
:104DB00000200B4902001870FEF760FA10BDC046D3
:104DC0004264FF1F2364FF1F93BA00112564FF1F75
:104DD0006709FF1F2B64FF1F6609FF1F6509FF1F7F
:104DE000AEDE000070B5134C142220001249FEF70D
:104DF0000BFB431E114D132B19D8AB78002B16D08B
:104E0000431C2B7009236B70002300190370287852
:104E10000B4B01302900C0B2187006F0E5FB297871
:104E200022000139C9B2002005F040FC70BDFFF737
:104E3000A1FFECE72564FF1FAEDE00002364FF1F27
:104E40004264FF1F10B5114B1A781870002A0ED05B
:104E500000280BD10E4B1A78062A07D85423D340CA
:104E6000DB0703D50B4B187802F072F810BD002851
:104E7000FCD0074B1B78012B02D0033B022BF5D84B
:104E8000044B0121187806F0FFFAEFE74664FF1F94
:104E90006D64FF1F6E64FF1F70B5504E504A51493C
:104EA0003070082005F08EFA0121092005F094F9F0
:104EB000092005F075FA0121002005F08DF9002088
:104EC00005F06EFAFEF714F906F0CEFA0322464911
:104ED0004648FFF735FF2D24030004221C70444987
:104EE0000130FFF72DFF30230470424D424C4370D8
:104EF00083702E3B062220004049EB87FEF784FAA0
:104F0000062813D0200006F06FFA022809D00321EA
:104F1000200006F0D9FA8D23E3706E3B237119331C
:104F20006371062220003549FEF7A8F9344B1B684F
:104F3000FC335C64FFF756FF0020FFF783FF314C22
:104F4000314A0121314B1278207801F0C3FF304AF9
:104F5000304B12780021207801F0BCFF01222E4B4B
:104F60001A702E4B5B78552B31D12D4B3B325A7238
:104F70002C4B2D4AAB81EA812B826A82202130782A
:104F800006F0F2FB0120404205F0DCFB012040422C
:104F900005F078FCFFF70AF9FEF7BEFE00F0AEFC64
:104FA00001204042FEF794FF012006F03DFCF02076
:104FB00001F04CF90121307806F066FA307802F001
:104FC00023F91A4806F028FCFEF754FD70BD642250
:104FD000174B5B7953431A000A32CBE74462FF1F39
:104FE000F94C00112D4D00118443FF1FE061FF1F9C
:104FF0000062FF1F0E43FF1F6509FF1FADAC0000DD
:105000009064FF1F6E64FF1F7842FF1F5942FF1F0D
:105010004264FF1F2364FF1F1464FF1F2462FF1FED
:105020001862FF1FC4090000CE0900004662FF1F7E
:105030002862FF1FF8B50A0020230D001A4019420C
:105040005DD05C4B1B78002B42D0FFF7F9FA5A4B2E
:105050005A4C5B4E99686268737A8A1ADB039A42EB
:1050600002D36160FEF706FD327A217A531EDBB26D
:10507000994230D1FFF75CF9637A002B25D0013BD0
:10508000DBB26372002B20D14E4B5B78552B01D1E4
:1050900006F09AFBE37A002B12D00023A27AE37287
:1050A0009A4202D0A372FEF773FD474A474F138816
:1050B000380001331380FEF767FE390006F034FA3A
:1050C000642370795843FFF7A5FD237A01332372D7
:1050D00020206840F8BD9142CED300272772FFF709
:1050E00061F9A37ABB4202D0A772FEF751FD374F98
:1050F0003800FEF749FE390006F016FABCE70BB29D
:10510000002B0ADA324B187806F036FC002801D062
:1051100006F0EAF980200002DBE70224214206D0F3
:10512000264B01201A72FFF78DFE2000D1E70B07F6
:105130001BD5FFF785FA204B2049214C98684A6817
:10514000637A821ADB039A4202D34860FEF792FC2C
:10515000FFF728F9FFF7ECF800F0EAFB2368DB071C
:1051600001D5FEF7ADFF0820B3E710230E001E4067
:10517000194209D0FEF70CFD0E4B1B78002B01D114
:10518000FEF7DEFD1020A4E70124214209D01148DA
:1051900000F06EF806F020FB3100092005F01CF845
:1051A000C3E7042408002040214200D192E7FEF723
:1051B000ABFEBAE74664FF1F3462FF1F1862FF1F91
:1051C0002862FF1F2462FF1F0C62FF1F5942FF1F4E
:1051D0004462FF1F3C42FF1FF0B51B4B1B4F1B8857
:1051E0003A8804001A4E1B4D85B09A420DD8328879
:1051F0009A420AD3184B1A882B889A4205D1174A2B
:10520000174B12881B889A421BD0052001F074F8B6
:105210003B8802AA13803388019053802B88114D5C
:1052200093800F4B02A91B88D3800F4B2A781888D4
:1052300002F090FD0D4B08212878019A1C7006F0B1
:10524000E3F805B0F0BDC0461264FF1F4E42FF1FD9
:105250004C42FF1F4A42FF1F1064FF1F0E64FF1FD6
:105260004842FF1F6E64FF1F5042FF1F0C64FF1F68
:1052700013B50C4B1C78002C11D1002801D00A4B1F
:1052800018600A4A0A4B11780A4A10780A4A0192B1
:105290000A4A0092002205F001F9200016BD1124EF
:1052A000FBE7C0466D64FF1F0864FF1F6C64FF1FAF
:1052B0005C64FF1F6E64FF1F4864FF1F4C64FF1F88
:1052C00010B5064B12201B78052B06D1044B132278
:1052D0001988044B187801F0EBF910BD6D64FF1FBD
:1052E0005042FF1F6E64FF1F10B500240122114BB6
:1052F00052421870104B1C70104B1A8001F084FF42
:1053000004220F4B21001A700E480C3206F0ECFA02
:10531000102221000C4806F0E7FA07220B4B1C6014
:105320000B4B1C700B4B1C700B4B1A700B4B1C70F7
:1053300010BDC0466E64FF1F6D64FF1F5042FF1F0B
:105340006C64FF1F5C64FF1F4C64FF1F4864FF1FF9
:105350002264FF1F2164FF1F5242FF1F2064FF1FB2
:10536000F8B5174C0600257806A814240078052DFA
:1053700023D1B41F134FA5B21824BD421DD88D1FD1
:10538000ADB2BD4219D8FA256D00AA4215D21D0052
:105390000D4F0A3DADB2BD420FD80C4C26800C4CCF
:1053A00021800C4900240A800B4A1380FFF714FF68
:1053B0000A4B0421187806F037F82000F8BDC046E3
:1053C0006D64FF1F790C0000750C00004E42FF1F3A
:1053D0004C42FF1F4A42FF1F4842FF1F6E64FF1FDF
:1053E000F0B50BB20D0089B0002B00DB70E1A44ECC
:1053F000307806F0C1FA041E50D00378A22B00D1F9
:1054000022E1D02B1AD0912B45D143780E2B42D1DB
:105410009C4B82889A423ED19B4A83681278052A27
:1054200039D1032018567F2835D0984B1B68002BA4
:1054300031D05B68002B2ED098472CE0807807286D
:1054400029D806F0D1F90428183F3F74A8D863780A
:10545000002B0CD101218C4B19708D4B1A78002A2E
:105460005BD08C4B307801F035FD002855D00722F9
:10547000854B1A7051E061780029F8D1E378002B50
:1054800011D0854A854B1278307801F023FD607089
:105490006378002BEBD1200006F026F88020000274
:1054A000684009B0F0BD784B1B78022BF3D0012186
:1054B000307806F031F90028EAD10121307805F082
:1054C000E3FFE5E76378002BD1D16F4F032807D1C5
:1054D0003B78052B02D101333B701EE00223FBE732
:1054E0006F4B1A886F4B0293002A0BD01B78002B4E
:1054F00003D00121307805F087FF3B78062B04D1DB
:10550000013BE9E7029B1A70F7E7042B41D1012127
:10551000029B3078197005F0B7FF5C4B1B68002BBD
:10552000B9D01B68002BB6D0574A107884E763784F
:10553000554F002B27D10622211D5B4806F00CFA9F
:1055400062895A4B5A491A80A2895A4B1A80E389B8
:105550000B800521397058490A80584A1380228AE5
:10556000574B1A80574B1B78012B09D11F2000F095
:10557000C3FEFA22920042430421307805F044FF32
:105580000022484B75E7312B00D070E70022454BD5
:105590001A700323A0E706220021434806F0A4F96D
:1055A0000023454A04211380444A30781380444A3A
:1055B000138005F039FF0821307805F035FFA37915
:1055C000083B5A425341304A03331370304B1B7827
:1055D000002B06D0334B30781A78002A06D001F021
:1055E000B7FC0122314B52421A8096E70121197013
:1055F00005F04AFFF5E70821307805F015FF6378DC
:10560000002B00D047E72C4B2D4F0293E388029AE2
:1056100004211380294B307803932389039A138044
:1056200063893B8006F078F8002800D033E7264BEA
:105630001B68002B00D12EE7039902983A8809884D
:1056400000881B68984726E74379132B00D022E790
:105650000389012B0AD11D4B1B78022B06D108218F
:10566000307805F0E1FEFFF72BFE14E7052000F08F
:1056700043FE08210200307805F0C6FE0BE7C04665
:105680006E64FF1F051400006D64FF1F0864FF1F98
:105690007842FF1F5942FF1F4264FF1F2364FF1F10
:1056A0004464FF1F4664FF1F1564FF1F5042FF1F25
:1056B0001C64FF1F1E64FF1F1264FF1F1064FF1F86
:1056C0000E64FF1F1464FF1F0464FF1F0C64FF1FA0
:1056D0008020C001014200D0E2E6CB0731D5324B39
:1056E0001B78002B1DD0314E05AC3378052B1AD119
:1056F000023B23702E4B21001B7823722D4B1B780D
:1057000063722D4B187801F089FB002809D007201F
:105710002A4B30701B68002B03D01B68002B00D075
:1057200098470120BCE60E20254B06221B78254910
:105730002370254B1B78637002ABC01806F00CF980
:10574000D8E7022308001840194209D0174B1B78EC
:10575000052B03D11D4B188805F076FF02209FE62C
:105760000424214203D0FFF737FD200098E60823E8
:1057700008001840194200D193E6154B1C78012C03
:1057800003D0022C0DD008208AE6124B124A13498E
:1057900013481B881288098800880094FFF7E0FDF1
:1057A000F1E7FFF78DFDEEE74664FF1F6D64FF1F15
:1057B0005242FF1F2064FF1F6E64FF1F0864FF1F1B
:1057C0002264FF1F5342FF1F2164FF1F5042FF1F2F
:1057D0000C64FF1F4842FF1F4A42FF1F4C42FF1F3D
:1057E0004E42FF1F10B502A804880B20002C10D1D8
:1057F000496808784978090201430C48814209D177
:10580000022119800A4B59881170DB7800205BB2A5
:10581000537010BD074C0A20A142FAD10221198011
:10582000034B998811705B79F0E7C0466E2A00003F
:105830000C62FF1F6F2A0000F7B5150008AA168832
:105840004A680F4F14785278120222430A24BA424F
:1058500014D10122DBB2019200962A0005F024FD4A
:10586000041E0BD1074B1B68002B07D068782A78E1
:105870000002104342425041013098472000FEBDD3
:10588000022900008064FF1F30B501250379040060
:10589000BFB02B4225D01449408805F071F828424A
:1058A0000CD0124B01A95B8D00220B8002234B8090
:1058B0000F4B5B888B80608802F042F90D4960884D
:1058C00005F05EF8C0070CD50B4B01A91B88002220
:1058D0000B8002234B80064B9B888B80608802F0F4
:1058E0002FF93FB030BDC0467864FF1F7C42FF1FD8
:1058F0000C62FF1F7064FF1FD642FF1F10B5074CDC
:105900000749200004F0F2FF2000064904F0EEFFF2
:105910000721054A054804F0ABFF10BDFFFF00005A
:105920007864FF1F7064FF1F20BB00117C42FF1FC3
:1059300010B5024802F086FF10BDC046895800111C
:105940000200F0B501270A480A4E51188B1A002BA5
:1059500000DCF0BD0824157843086840384040005A
:10596000805B013C58406D08002CF5D10132EDE719
:10597000FFFF00003ABB0011F0B500250F269D4245
:1059800000DBF0BD4C5D070944403440A400A05842
:1059900001357840F3E70000F0B589B06A460D00A4
:1059A0000B000F27110010351C7801332600240945
:1059B0003E40167054700232AB42F5D12023024AA9
:1059C000FFF7DAFF09B0F0BD40BB0011F0B54E782B
:1059D0000B7889B036020C00170001901E43012A93
:1059E00061D9954B9E4200D877E001339E421CD18D
:1059F000062A17D1CA788B7812021A430B791B0436
:105A000013434A7912061A438C4B5A6100221A70CA
:105A10005A808B4A5A608B4A9A608B4ADA6000201F
:105A200009B0F0BD88225205EEE7884B9E423CD17A
:105A300082498B78002B00D0F6E00C2A31D10F225E
:105A4000A3789343E278120213432279120413439A
:105A50006279120613434B60E279A0791202024385
:105A6000207A00041043627A12060243CA60E27A86
:105A7000A07A1202024376484A81834208D804235E
:105A80006E49142201980B7005F066FF1420C7E7D9
:105A90001201D21889235B059A42F0D801238B703A
:105AA000BDE7022AFAD00523EAE76A4A01239642B3
:105AB000E6D1FFF705FC052F0CD9E378A2781B028D
:105AC0001343227912041A4363791B061343624A73
:105AD0000393136005F078FEA1E7584D2B78002B57
:105AE0009DD1AB78002B00D1A0E02B8901339BB274
:105AF0000093B34200D091E0132AD4D9CF7C8B7CA1
:105B00003F02122120001F43FFF71AFF874200D0F7
:105B10008EE0002E3DD1E378A2781B021343227958
:105B2000E96812041A4363791B06134303930A229C
:105B30008B4212D1FF23A370E370237163716B89D1
:105B4000002B09D1E37B227C1B0212041343A27BAE
:105B500013431B0901336B8100226B89002B8ED00C
:105B6000002A67D1686837013818000B6B69000399
:105B70000390984205D9686105F016FEEB78013371
:105B8000EB7068681022A11C381805F025FC2E81E6
:105B900045E76F89009A7B1E9BB293423AD1E27827
:105BA000A37812021A43237905A81B0413436279D0
:105BB0006C6812061A43EB6800920392211D0C22B6
:105BC000049305F0C9FE0120260004A940421036C6
:105BD000FFF7E2FE013F012F17D1009A0B23286146
:105BE000824200D04CE704221C49200005F0F4FB5F
:105BF000042203A9686805F017FDE968039AFF23EA
:105C0000914200D13CE7F73B3AE73100FFF7C4FE91
:105C10001036DFE70923B742A4D831E7009BB3422F
:105C200000D9FCE607232BE7022329E7032327E714
:105C3000062325E70A2323E7FFFE0000F042FF1FAB
:105C400000000111FFFF00005048593601FF00001D
:105C5000FFFF001102FF000034F00040FC42FF1F74
:105C600010B5034C0B000122210000F06BFA10BDAF
:105C7000215E00110B8870B506000D000224162B62
:105C800011D92B000322094900F05CFA041E0AD145
:105C9000074B2A881B88191C934200D9111C30001D
:105CA00089B200F0EFFA200070BDC0464D5E0011D1
:105CB0009664FF1F10B54A780400013A0B000220D9
:105CC000012A07D80A78002A04D0052220000249B8
:105CD00000F038FA10BDC0467B5E00110A7810B59E
:105CE0000B0004000220002A04D0072220000249F1
:105CF00000F028FA10BDC046275F00110A7810B5E1
:105D00000B0004000220002A04D0092220000249CE
:105D100000F018FA10BDC0468D5F001110B5034C9D
:105D20000B000B22210000F00DFA10BDBD5F001129
:105D300010B5034C0B000D22210000F003FA10BD3A
:105D40002F60001110B5034C0B000F22210000F052
:105D5000F9F910BD896000110A7810B50B00040034
:105D60000220002A04D011222000024900F0EAF9A2
:105D700010BDC04699600011002310B51322190010
:105D800000F0E0F910BD000010B5034C0B00172225
:105D9000210000F0D7F910BDEB600011002310B511
:105DA0001922190000F0CEF910BD000010B5034C07
:105DB0000B001B22210000F0C5F910BD2561001168
:105DC000F7B584890D0006000121002C22D00023A4
:105DD0008268D3561778002B1EDA0C2C1AD90C3C8B
:105DE000A4B2131940880093230002F086FE431EDC
:105DF000984101307B06DB0F6B703F23013C1F4055
:105E0000A4B22870AF70AC80002C07D0B368013307
:105E1000AB6000210800FEBD0020EBE7AC60F8E7B6
:105E20000B7803704B8843704B881B0A83700B7987
:105E3000C370042070470420022B06D10020537841
:105E400011781B02009A0B43138070470B88037074
:105E50000B881B0A4370022070470420009983427C
:105E60000AD1537810781B0203430B80D3789078C3
:105E70001B02034300204B807047F8B50D004B78A0
:105E800001240021461C03702B788B4201D820008E
:105E9000F8BD6B78B01C4F1C012B10D1890069181C
:105EA0004B88022233704B88B9001B0A7370691843
:105EB00005F08AFB04360434A4B2F9B2E4E71223F5
:105EC00059436B185A88043132705B8810221B0AC0
:105ED0007370691805F078FB12361234ECE770B570
:105EE000049D14001E00052B01D8042070BD6378AA
:105EF00012781B0213432B80E378A2781B02134312
:105F000002226B802A71211D681D063E05F05CFB94
:105F1000B2B22A81E92AE8D82800A11D0A3005F08A
:105F200053FB0020E2E7002310B50A789A4201D81B
:105F3000900010BD9A008A18548801330470548868
:105F4000DBB2240A4470948884709288120AC2706A
:105F50000430EAE710B51100029C062B04D004209F
:105F60001022142B01D010BD022222714B78087828
:105F70001B0203432380CB7888781B020343638092
:105F80000431601D05F020FB0020ECE710B50C7813
:105F90008B7804315C43E4B203702200013005F0D9
:105FA00013FB601C10BD0420022B06D10020537887
:105FB00011781B02009A0B431380704710B50C0038
:105FC0000A88023105F000FB208810BD70B504007E
:105FD0000D0004981100012B01D8042070BD167823
:105FE00052781202324302800200F132557014706E
:105FF000E125002C00D10C35023B9AB24280AA4226
:10600000EBD80231043005F0DFFA0020E6E7042087
:10601000009983420AD1537810781B0203430B8006
:10602000D37890781B02034300204B80704710B553
:106030000C000A88023105F0C7FA208810BD000064
:1060400070B501211E000420049C0E400B4218D1A3
:10605000CB40DDB28D4214D90A49DBB2098899429E
:106060000FD32300EE331D70330058001118497808
:10607000165C0902314301332152D9B28D42F4D862
:10608000002070BD0843FF1F10B50C000A880231C4
:1060900005F09AFA208810BD10B50C788B78043181
:1060A0005C43E4B203702200013005F08DFA601CFD
:1060B00010BD10B511000298032B01D8042010BDAB
:1060C00014785278043B120222430280CA788C78FA
:1060D0001202224342809AB28280EB2AEED8043127
:1060E000063005F071FA0020E9E710B50C000B88C6
:1060F00003700B881B0A43704B8883704B881B0A04
:10610000C3708A880430063105F05EFAA088043036
:1061100080B210BD0420012B03D100201378009A17
:106120001370704710B50C000B8803700B881B0AA6
:1061300043704A880230043105F046FA6088023024
:1061400080B210BDF0B589B003931E4B029242009D
:106150000700D05A019102F020F81325061E2DD019
:10616000029B01240370019B002B04D000190399AA
:106170009847001984B26B461B7A5BB2002B0FDA8A
:106180001021380002F01CFB1925002813D1300023
:106190003219E1B202F066FC051E0CD10C34A4B237
:1061A000042304AA380005A993800696948101F07F
:1061B000AFFD051E02D0300005F096FA280009B0A8
:1061C000F0BDC0469464FF1F70B505000C000028A8
:1061D0000CD00020814209D010222000044905F093
:1061E000F3F901202B7823736B78637370BDC0467D
:1061F00080BB0011F0B506000D0017001C0085B033
:1062000002291BD00020102907D1022B07D0102B08
:1062100003D115E00020102C08D005B0F0BD694670
:106220003800FFF7D1FF2A0069460BE069463000CD
:10623000FFF7CAFF22006946380004E0022BE9D1CB
:106240002A003900300005F02FFAE6E7031CF02899
:1062500000D9F023032008499AB2013A0B80D317E2
:10626000034006499B189B100B80D30F04499B18D1
:106270005B100B807047C0460C43FF1F0A43FF1F93
:106280000843FF1F034B1B888B4202D3024B400085
:10629000C15270470C43FF1F9464FF1F014B400025
:1062A000185A70479464FF1F1722014B1A807047D9
:1062B0009464FF1F70B505000E2005F01DFB041E41
:1062C00013D0D02303700023062283700749457042
:1062D000033005F079F9064B2100DA8A62811B7ED2
:1062E0002373044B187805F047F970BDB064FF1FA5
:1062F000A064FF1F5C43FF1F262803D8024B400009
:10630000C05A70470148FCE70E43FF1FFFFF000023
:1063100070B506000C00094D1C220021280005F074
:10632000E3FA074B1E70074B1C7005F095FA01232A
:10633000002801D0002312202B7070BDA064FF1F25
:106340005C43FF1FC164FF1F70B505000D4C0800C2
:10635000E260A16010220021656005F0EDFA0128DD
:1063600003D11021A06802F058FD1022002128005E
:1063700005F0E2FA012803D11021606802F04DFD1A
:1063800070BDC046A064FF1F70B5041E05D1002972
:1063900003D006220D4805F017F90D4B1D78012D8D
:1063A00011D1002C05D102221A7005F0F5F9280050
:1063B00070BD00221A70074B1B78FF2BF7D020000E
:1063C000FFF778FFF3E70025F1E7C046B064FF1F51
:1063D000A064FF1F5C43FF1F030010B5002801D11C
:1063E000002010BD00780B4A002803D15988D182C3
:1063F0001B7913761378022BF2D10023984200D137
:1064000003331370044B1B78FF2B01D0FFF752FFAF
:106410000120E6E7A064FF1F5C43FF1F002911D0A5
:1064200000280CD04B79012803D14022524213435B
:1064300003E03F221340032802D001204B71704734
:106440004022F4E70800FAE770B5094D010028780A
:1064500000280BD0074C0622200005F0B5F82100DB
:106460002878FFF7DBFF200005F026F870BDC04656
:10647000C064FF1F9A64FF1F00290AD0012808D1B9
:106480003F224B799343C02B03D0403B5A425341A8
:10649000981C704770B5174D06002B78FF2B15D050
:1064A0000A2005F029FA041E10D0D0230370C83B3F
:1064B0008370114B11491B784670C370062204305B
:1064C00005F082F82100287805F056F80C4B1B786F
:1064D000012B0DD10B4B1B68002B03D09B68002BAD
:1064E00000D09847084B04211878084A05F0CCF8EA
:1064F00070BDC0465C43FF1FC064FF1F9A64FF1F4E
:10650000BC64FF1FE864FF1FEC64FF1F60EA00002B
:10651000014B98687047C046A064FF1F014BDB68C1
:1065200018687047A064FF1F074B10B5DA6813683E
:1065300001331360054B1878FF2803D08021C9016F
:1065400004F0A2FF10BDC046A064FF1F5C43FF1F04
:10655000F7B50E0002F0C8F8051E1CD00E4B0662FF
:106560001F78002F00D10778AB791020019305F038
:10657000C3F9041E0FD0D0230380C73B8370019B57
:10658000E91DC3700622043005F01EF82100380012
:10659000E66004F0F1FFF7BD5A43FF1F014B187886
:1065A0007047C046C064FF1F054B002805D1054B4E
:1065B0001A78054B002A00D1014B18007047C046DD
:1065C000B064FF1FC064FF1F9A64FF1F014B58682F
:1065D0007047C046A064FF1F024B1868431E9841D5
:1065E000C0B27047C464FF1F421E03000120152A79
:1065F00003D9FF3B5A425341D8B27047F0B51C0053
:1066000000230E0085B0039002920B70029A934211
:1066100001D3002019E0E55C5A1CD2B2002DF8D05D
:10662000029851198142F4DC0233DFB2A35C1800F6
:106630000193FFF7D9FF002807D0013D019A039984
:10664000EBB233708A4202D1E01905B0F0BDDB191C
:10665000DBB2DBE710B50C0002F09EF8030012205D
:10666000002B03D02100588805F026F910BD00004A
:1066700070B50E4D84006359002B15D0186A0028A0
:1066800001D005F029F92B59586A002801D005F0EE
:1066900023F92B59986A002801D005F01DF92859D3
:1066A00005F01AF900232B5170BDC046D064FF1FBE
:1066B0001C4B70B504000E00150099420AD11A4B0C
:1066C0001B68002B01D1122070BD1B68002BFAD073
:1066D0009847F9E7154B994215D1134B1B68002BCE
:1066E0000AD01B68002B07D09847002804D1104B14
:1066F0001C70104B1D70E7E729002000FFF7AAFF70
:106700000028E1D1F3E7080001F0EEFF0028DAD01D
:1067100003780320A342D7D12900300005F0CCF83C
:10672000D2E7C046FEFF0000CC64FF1FFFFF000061
:10673000C964FF1FC864FF1FF7B50400808801F01B
:10674000D3FF0025A84203D00578A08802F008F8FE
:106750001C4E3378002B1FD0AB421DD11A4B2800A2
:106760001978FFF777FF002818D000233370A3793A
:106770000820A778A688019305F0BEF8011E0DD069
:10678000D0230370CA3B8370019B4770868083715E
:10679000280004F0F1FE01E0002DE8D1A0880B4BA9
:1067A0008200D358002B01D0FFF762FF1721A08889
:1067B000FFF768FDA08801F027FDA08801F0FEFD2D
:1067C000F7BDC046C964FF1FC864FF1FD064FF1F28
:1067D000F0B587B01D000CAB1B88070001930DAB13
:1067E0001B88142002930EAB1B88160003930FAB7B
:1067F0001B880091049310AB1B88059305F07CF86F
:10680000041E1AD0D0230370CB3B47708370C67030
:10681000062229000430002D11D004F0D5FE019B82
:1068200021006381029B0098A381039BE381049B69
:106830002382059BA37404F09FFE07B0F0BD05F012
:1068400053F8ECE7F7B5009308AB1B8807000C2062
:106850000D001600019305F04FF8041E13D0280018
:1068600001F042FF00280FD00078D0232370C93BED
:10687000A370009B21002381019B6770A580E680A7
:10688000638104F079FEF7BD014B1878EDE7C0464F
:106890005C43FF1F13B5040064890389C2888188A3
:1068A000C0780094FFF7CEFF13BD000010B5044C74
:1068B0002068002803D005F00FF80023236010BDE6
:1068C000D464FF1FA122F0B5818892004A43384B5F
:1068D000384F1B6804009B189D2292009B188279F8
:1068E00089B01A603B68002B5FD01D78324B1B6863
:1068F000002B04D05B68002B01D0002098472600B5
:1069000008363100E079FFF7B7FD237DE071020022
:10691000E0780493638A29000393238A0293E3892E
:106920000193A38800933300FFF752FFE378002B15
:106930000BD1E289A379A18802920196E27928001D
:106940000092012201F0DAFEE0703B68002B20D0BB
:10695000FFF7ACFF194D287800281AD0184B19788A
:10696000FFF778FE002814D02B78E67808200793EC
:10697000A78804F0C1FF011E09D0D0230370CA3BD1
:106980004670837087808671079804F0F5FD0023B8
:106990002B701721A088FFF775FCA08801F034FC4C
:1069A000A08801F00BFD09B0F0BD064B9DE7C04685
:1069B0003409FF1FD464FF1FE864FF1FC964FF1F71
:1069C000C864FF1F5C43FF1FF8B5070008000E00F6
:1069D00001F08AFE041E18D02620FFF78DFC051E4C
:1069E00000D12578062004F087FF041E0DD0002179
:1069F000062204F079FFD0232370C23B2100677088
:106A0000A370A680E8B204F0B7FDF8BDF0B585B07C
:106A100001930AAB1B78070002930BAB1B780800AD
:106A20000D000092039301F05FFE061E22D010209D
:106A300004F062FF041E1DD01022002104F054FF58
:106A40002620FFF759FC002800D13078D02323708E
:106A5000C13BA370009B21002372019B677063728E
:106A6000029BA580A372039BC0B2E3720C9BE36000
:106A700004F082FD05B0F0BDF7B50D00019001F006
:106A800033FE071E20D00E2004F036FF041E1BD05C
:106A90002620FFF731FC061E00D13E78D02323804C
:106AA000C53B0622A370F91DE01C04F08DFD019B7F
:106AB0002A0063810123DD401A401D40210022731A
:106AC0006573F0B204F058FDF7BD0000F0B585B075
:106AD000029010000D0017000A9E039301F004FEBF
:106AE000041E31D0029B002B2ED1039B02795B0741
:106AF00024D5122313430422002E08D10B99002918
:106B000005D10C99002902D10D9900291AD01A43F8
:106B10000D9B2271002B00D0C9E0002E00D1CFE0E8
:106B2000002D00D0CCE0606A002801D004F0D4FE33
:106B30001C21300004F0B8FE606205E002239A4395
:106B40000E33D7E793432371654BBA00D458002C1A
:106B500000D1AAE0002E10D0236A002B03D11C2004
:106B600004F082FD20625E4BBA00D358186A0028F8
:106B700003D01C22310004F027FD0C9B002B12D007
:106B8000574CBB001D596B6A002B03D1162004F033
:106B90006BFD6862BB00E358586A002803D01622D8
:106BA0000C9904F011FD0D9B002B11D04C4DBC0035
:106BB0006659B36A002B03D1142004F055FDB0626E
:106BC0002B59986A002803D014220D9904F0FCFC7C
:106BD000380001F089FD051E67D0414BBA00D3583B
:106BE000002B62D01A6A3420002A00D11C389A6A1D
:106BF000002A01D0143080B20B9A002A01D01C3038
:106C000080B25B6A002B01D0163080B204F074FEB3
:106C1000041E4AD01822002104F066FE2620FFF749
:106C20006BFB0190002801D12B780193D0232370B6
:106C3000029B200063700A23294EA370039BBD00B2
:106C4000A371AB59A780196A1830002905D01C22FE
:106C5000A06004F0B9FC200034307359996A00290F
:106C600007D0030014221433E060029304F0ACFC5C
:106C700002980B9B002B08D003001C221C330B999D
:106C80002061029304F0A0FC02987359596A00290C
:106C900003D01622606104F097FC6B46210018793E
:106CA00004F06AFC3800FFF7E3FC05B0F0BD1022E9
:106CB0000D9B0D991B69A018236204F085FC2CE73D
:106CC0000B9B002B00D13FE7012D00D03CE7606A11
:106CD000002801D004F000FE1C210B982AE7C046D2
:106CE000D064FF1F10B5044C2068002803D004F0C6
:106CF000F3FD0023236010BDC464FF1F0B4B07B5D9
:106D00001A68002A01D100200EBD6946531C0120DB
:106D100012780731FFF772FC0028F4D002780123C3
:106D2000100018401A42EED0EEE7C046E064FF1FA4
:106D3000F0B51F4F01203B6887B0002B25D09B7812
:106D4000059300F0B3FB002821D00A20FFF7D4FA06
:106D500004000B20FFF7D0FA164B05001E78731EB7
:106D60009E413B68F6B2191DD878FFF757FB3B6888
:106D70002900DA7A043303929A79019302920090FF
:106D800033002000059A04F0D7FC07B0F0BDFFF7F0
:106D9000B5FF002805D00620FFF7AEFA0400072053
:106DA000D8E70820FFF7A8FA04000920D2E7C04678
:106DB000C464FF1FC064FF1F70B50A4E040033781F
:106DC0000D00FF2B0DD0042004F096FD011E08D00D
:106DD000D0230370CE3B45708370C470307804F0CC
:106DE000CBFB70BD6C43FF1F70B5040006200D0087
:106DF00004F082FD011E0AD0D0230370CD3B8370C6
:106E0000054B44701B688580187804F0B5FB002C96
:106E100001D0FFF767FF70BDC464FF1FF8B5264FB0
:106E200006003B680D001124002B05D10522234BE1
:106E30001B78134202D112242000F8BD204A1024EE
:106E40001268002AF8D01278002AF5D0DB0719D58D
:106E50002B789A1E012A1AD80C2004F005FC132462
:106E600038600028E8D000230A2243702900067009
:106E7000023004F0A9FBFFF75BFF041E0AD0FFF706
:106E800031FFD9E700F012FB0028E1D1E4E7002B45
:106E9000E2D0D0E70B4B1B78032BCDD11D20FFF7A1
:106EA0002BFA094B18800028C6D0084B042118780B
:106EB000074A04F0E9FBBFE7C464FF1FC164FF1F7A
:106EC000E064FF1FC064FF1FBE64FF1FEC64FF1F70
:106ED00060EA0000F7B50193194B14001A780523F6
:106EE00006000F0012201A4221D0012920D1154B93
:106EF0001D68002D1BD002201F2C18D8002C02D09A
:106F0000019B002B13D0104B1F221E706E1C002102
:106F1000300004F0E9FC01992200300004F054FB39
:106F2000310020002C70002F06D004F06DFCFEBD57
:106F3000064B12201D68DCE704F056FBF7E7C0465D
:106F4000C164FF1FE064FF1F6C43FF1FDC64FF1F71
:106F5000F8B50F4E12243368002B17D01B780F3C66
:106F6000834213D100250B4F0221387804F05CFADC
:106F7000094B042138781D8004F056FA074B28008D
:106F80001D8033685C7004F0DFFA04002000F8BD57
:106F9000C464FF1FEC64FF1FD864FF1FBE64FF1FA3
:106FA00070B5012823D11B4C2388002B03D01A4A2B
:106FB0001578002D07D0194B1B68002B02D01878CC
:106FC000FFF7C6FF70BD3B2B02D93C3B2380F9E79E
:106FD000134E0221307804F027FAFA222388920017
:106FE00002215A43307804F00FFA2580EAE70B4B70
:106FF0001B68002BE6D00B4B1B785B07E2D5084BD8
:107000000221187804F010FA0022024B1A80FFF7D0
:1070100069FED7E7D864FF1FBC64FF1FC464FF1F6D
:10702000EC64FF1FC164FF1FF8B51E4D28680028DF
:1070300003D004F051FC00232B601B4E3068002865
:1070400003D004F049FC00233360184F05243B783B
:1070500018002040234221D0154800F02BFA3B783D
:10706000234213D0202004F0FFFA2860002813D018
:107070002022002104F038FC202004F0F5FA041E40
:10708000306005D02022002104F02EFC002004E016
:10709000286804F021FC2C601320F8BD00F00AFAE7
:1070A000F4E7C046E064FF1FDC64FF1FC164FF1FFC
:1070B0006043FF1F10B50A4C23681A1E0ED000282B
:1070C00008D10130587004F03FFA002805D0236839
:1070D000002B02D00021FFF787FE0122100010BD17
:1070E000C464FF1FF7B5274E050033680191181ED1
:1070F00021D05C78244F012C30D1FFF7FFFD002810
:1071000025D02000FFF7F8F80400412814D91F4BC0
:10711000022118781E4A04F0B7FA1E4B3C3C1C8032
:10712000022233685A703B78002B14D12800019951
:10713000FFF75AFE0120FEBDFA2292004243002AC8
:10714000EED0124B0221187804F05EF9E8E7FFF761
:10715000D3F80200F3E700233B70EBE73B78002B0A
:10716000E8D1032004F0C8FB011E08D0D02303702F
:10717000CC3B457083703368187804F0FDF9FFF755
:10718000B1FDD7E7C464FF1FBC64FF1FEC64FF1FA1
:1071900060EA0000D864FF1F10B517498388020019
:1071A0008B4220D011D815498B4217D014490020AA
:1071B0005B1899B2012907D8926811785A42534155
:1071C000D8B2FFF7F9FD012010BD0E4A00209B1830
:1071D00007229BB29A424041C0B2F5E78368187813
:1071E000FFF768FFF0E7836899785A780902187802
:1071F0001143FFF777FFE7E70A20000006200000B1
:10720000F8DFFFFFAFDFFFFF014B18707047C0468C
:107210006D43FF1F10B5064C207001F041FA207835
:1072200004F0FAF90521207800F062FD10BDC04697
:10723000EC64FF1F0BB273B50D00002B00DBC4E044
:10724000884B187804F098FB041E0ED00378912B1D
:107250000FD0A22B00D1A1E0834B1878FF2852D089
:10726000210004F089F900284DD1802000026840F7
:1072700076BD43780F2B76D013D8052B70D00E2B0C
:10728000EAD18088794B98422BD8794B98421BD809
:10729000784B9842E0D1A3681878591CFFF774F82E
:1072A00038E03E2BD8D18378032B74D06CD8012BD7
:1072B0006ED0022BD0D1704B1B68002B23D05B68A3
:1072C000002B20D098471EE06C4BC0180C28C3D868
:1072D00004F0C2F81DC2C2150BC20B0B0B3223C245
:1072E0003C00674BC0180728B6D8664B1B68002BBC
:1072F00009D01B68002B06D0200098470AE0A3683D
:107300001878FFF7C7F8200004F0EEF8ADE7A068A2
:10731000FFF762F800289FD0F5E7A3681B78002BE1
:10732000F1D0554B1B68002BEDD01B68002BEAD029
:10733000210055489847EDE74F4B1B68002BE2D0E2
:107340001B68002BDFD021005048F3E7504B1B682F
:10735000002BD8D05B68002BD5D021004348E9E74B
:10736000FFF7EAF9CFE780884A4B984203D04A4BAF
:10737000984200D070E7464B1B68002BC3D05B6877
:10738000002BC0D02100D5E7153B012BBBD963E70B
:10739000FFF798FAB7E7FFF77DFAB4E73F4B1B78A2
:1073A000042B07D100236A4613800179408800F03E
:1073B000C5FCA8E7364B1B68002BA4D05B68002BEC
:1073C000A1D00100364898479DE7012421420AD008
:1073D000294B1B68002B04D05B68002B01D00020D8
:1073E0009847012043E78B070AD5264B1B68002BE3
:1073F00004D05B68002B01D020009847022036E7BC
:107400000421280008400D4200D131E7254E338881
:10741000002B21D0013B9BB23380002B1AD1FFF708
:10742000DBF800280AD0204B1C70164B1B68002B81
:1074300004D05B68002B01D020009847FFF7C6F806
:10744000694601F001FD6846FEF7FEFF1D20FEF7CC
:1074500053FF308004200AE7024B187803F0E4FF62
:10746000F8E7C046EC64FF1F6D43FF1F0E200000CD
:107470000120000009100000E464FF1FFEDFFFFF91
:10748000AFDFFFFFE864FF1F0C2000000B200000AF
:10749000CC64FF1F0D20000013200000C164FF1FFB
:1074A000FFFF0000BE64FF1FBC64FF1F10B501F0AA
:1074B0009BF910BD014B18607047C046E864FF1F80
:1074C0000B880020162B01D817230420014A1380B3
:1074D0007047C0469664FF1F00207047074A0300AC
:1074E0001188814207D091880020994202D1013051
:1074F0008000101870470020FAE7C046F464FF1FB0
:10750000F0B58F7806000D00C5B01E2F15D1FFF71E
:10751000E5FF051E03D10024200045B0F0BD002288
:107520003B003100C078009200F0B2FB0400A81CC0
:1075300000F0D2FBFF23EB70EEE7264B062403930B
:107540001B78FF2BE8D0182FE6D87B08224A013B96
:10755000DB0002929A589446002ADDD0029AD31892
:107560005B68002BD8D00878002802D14B78012B1B
:1075700002D10624122FCFD107AFAB8869780097CC
:107580006446AA68A047041EC6D1AB78029A5B087D
:10759000013BDB00D318390030005B689847041EBC
:1075A0000BD1AB78042BB6D0039A310010782200AF
:1075B000009700F06DFB0400AEE76A78002AABD1BB
:1075C000AA7805A93B88087130000A704B80FEF745
:1075D00047FBA0E77043FF1F90BB00111D4B37B561
:1075E000050098420BD000290AD1FFF777FF002849
:1075F00005D11948FFF772FF002800D0058037BD7C
:1076000001291AD1FFF76AFF041EF8D001235B425B
:107610000380A378FF2BF2D0FE2B07D00023E07865
:107620001422009329001E3300F032FBA01C00F04E
:1076300053FB01235B426380E1E70229DFD101397B
:1076400001F0BEF80028DAD12800FFF747FF041E3A
:10765000DFD1D4E7FEFF0000FFFF0000022210B5DB
:10766000074B52421A80074801325A809A80DA80CA
:1076700000F07EFA044801F025F8002010BDC04655
:10768000F464FF1F01750011DD7500110388F7B563
:107690000400002B02D102252800FEBD4268022111
:1076A000137825485268FEF7A5FD00282ED0234FF9
:1076B00001253A88002AEFD0802321885B0201252A
:1076C0009B1A9942E8DC0C2003F0CEFF061E31D055
:1076D0003B8822889C4600231800019561469DB294
:1076E000491989B2AA421BD8002801D062443A80C5
:1076F00000233000082208C0210003F065FF104A73
:107700001368002B13D100251660C5E762680221BB
:1077100013780C485268FEF76DFD0028C7D1BAE710
:1077200060681D014019418101330198D6E71A00B4
:107730001B68E6E71325AFE7FEBB00116E43FF1F92
:10774000F064FF1FFCBB0011014B18707047C0466E
:107750007043FF1F14230A0010B51A40194204D0C9
:107760000122102101F048F810BD4B06F9D4012088
:1077700088434000F8E710B514008B0604D50122B9
:10778000102101F039F810BD08230A001A401942EF
:1077900002D14BB2002B0FDA102101F02DF8002896
:1077A00008D02300F2331B78002BECD0F13423787F
:1077B000012BE8D10020E6E703208907FAD4E2E7AD
:1077C000F0B51F00184B85B01C6801900291039220
:1077D000002C27D1200005B0F0BDA5683301ED18BD
:1077E0006B89019A934211D3029A93420ED8002FCB
:1077F00004D10A9B002B10D12C00EBE73B00297829
:10780000039A6868FEF7F6FC0028F2D10136B6B29A
:10781000A388B342E1D82468DAE7A3680A9A5B89AF
:107820001380E9E70026F3E7F064FF1F37B50C008B
:107830000A8849880123914217D3002A15D0651D73
:1078400023792A0002210A48FEF7D4FC10230028DD
:107850000BD023796188208800242A000094FFF748
:10786000AFFF0A23A04200D0230018003EBDC0464F
:10787000FEBB001113B50A0008884988012388421D
:107880000BD8002809D00024137905320094FFF7A3
:1078900097FF0A23A04200D02300180016BD13B59D
:1078A0000A0008884988012388420BD8002809D09B
:1078B0000024137905320094FFF782FF0A23A042C7
:1078C00000D02300180016BDF0B58BB003904A8895
:1078D00008880E000123824255D3002853D000238C
:1078E000012704AC23700022718813000092FFF777
:1078F00067FF051E3ED02078002835D12B78022B5B
:1079000018D167706A8983000130E31880005A80BB
:1079100069680222201803F057FE23780133DBB296
:107920002370042B19D93B006889013080B2002BE9
:10793000D9D01FE002236370122358436A892318A9
:1079400004305A8069681022201803F03DFE237825
:107950000133DBB22370002BE5D10C4A6B899B18F5
:107960005A425341DBB2DFE76378012BE4D12B7835
:10797000022BC7D022780A23002A04D021000398C2
:10798000FEF798F9002318000BB0F0BD0100FFFFCF
:107990000F4BF0B504001868002816D083685D8985
:1079A000A54207D88288AE18B44203DA12019A18A9
:1079B000934201D10068EFE71E005F891036A742AD
:1079C00004D1002900D00D801800F0BD3300EFE78E
:1079D000F064FF1F70B505000C0008880021FFF758
:1079E000D7FF03000120002B04D022002800197AC1
:1079F000FFF7C1FE70BDF7B50C0000250190230014
:107A0000EE331B78AB4201D800200AE06B00E65A47
:107A100000213000E718FFF7BBFF002802D12680C5
:107A20000130FEBD017A0198FFF794FE002802D0D4
:107A30003B882380F5E70135EDB2E0E710B504009F
:107A400008880021FFF7A4FF03000120002B03D0CA
:107A50002000197AFFF77EFE10BD0000054B1B6861
:107A6000002B01D1180004E09A6852898242F6D1B5
:107A700098887047F064FF1FF0B50E27002687B086
:107A8000039302ABFF183E8005001F4B4089140092
:107A9000984207D02B78013000976A6880B2FFF7D0
:107AA0008FFE060002212B7818486A68FEF7A2FBB9
:107AB00000280FD06C892000FFF7D0FF002802D0EB
:107AC000013C0419A4B2039B002B00D01C803000A1
:107AD00007B0F0BD02212B780D486A68FEF78AFBDB
:107AE0000028E7D102212B780A486A68FEF782FB5A
:107AF000002807D0002EDED03B88A342DBD174895A
:107B0000013CDFE76C89DEE7FFFF0000FEBB0011F0
:107B1000FCBB0011FABB001110B50C00FFF7DEFC36
:107B200003000220002B0AD0002C00D023609B7899
:107B30001720FE2B03D00138FF2B00D1002010BDF1
:107B400073B50D0001A904001600FFF7E5FF172823
:107B500005D0002E04D129002000FEF727F976BDBC
:107B600001221021200000F047FE0028F3D0F6E7A4
:107B7000014B18607047C0460065FF1F37B56B4664
:107B80009D1D010004000222280003F0E5FE2B8861
:107B9000B02B0ED12379122B09D12300FA331B7895
:107BA000012B06D10121608800F0E0F801E01B2BD9
:107BB000F8D037BD10B5054B0421187000F098F8C7
:107BC000FFF74CFDFEF770FB10BDC0460465FF1FBC
:107BD0000020F0B50BB20F0087B0834234DA274B98
:107BE000187803F0C9FE051E2BD00378A02B25D1F1
:107BF00003AE3100FEF7E4F8041E0BD1B378DB07C7
:107C000024D51F4B06341B68002B03D03100688835
:107C100098470400A868002801D003F065FD002CF7
:107C200008D1184A039B1340174A934206D0B378F1
:107C30001B2B03D00121688800F098F8280003F07E
:107C400053FC80200002784007B0F0BD0F4B1B684A
:107C5000002B10D0310068889847041EDAD0737862
:107C6000002BD7D1B27801A90A704B800C716888BB
:107C7000FDF7F6FFCEE70624F1E7C0460465FF1FD7
:107C8000FC64FF1F00FFFF00000112000065FF1FE2
:107C9000F7B50190FC200D0017001E0003F02CFE2C
:107CA00004001320002C12D0B02320002370089B66
:107CB000F4226770658026710830002B08D0190007
:107CC00003F082FC2100019803F056FC0020FEBD69
:107CD000089903F009FEF5E710B5041E06D00078F8
:107CE000FD2803D803F0F8FBFF23237010BD00002C
:107CF0000A1F93B210B504000220032B05D882405E
:107D00000020024BD1529B189C7010BD2465FF1FB0
:107D10000B8870B5043B04000D000220032B0BD828
:107D20000121200000F04CFD03001420002B03D0A3
:107D30002900200000F0DEFB70BD000007B5130035
:107D4000034A00920A00012100F02CFC0EBDC0463F
:107D5000797F001107B5019203220092024B0A00BD
:107D6000122100F049FC0EBDF77F001107B56B46EC
:107D700001AA11800449D88008780633012802D16D
:107D8000190003F0A1FD07BD0565FF1F0C4B10B5E1
:107D900018700023FF210B4A138013819381938075
:107DA000094A53801370517293819372D174D382B4
:107DB0001375517703F0A0FC00F0FCF910BDC0462C
:107DC0003465FF1F2465FF1F0665FF1FF0B58DB0EA
:107DD0006B46002003910C229B5E834200DBB0E0E7
:107DE0005D4B187803F0C8FD051E00D1A4E00378B0
:107DF000902B00D09DE006AF01004688380000F0CF
:107E000013FA79680400002900D19CE03B88052B17
:107E10006ED13B89032B1CD905AC200000F0A2F8E1
:107E20006288172A61D83989131D994231D179683E
:107E3000237804310291D90738D5607800F08EF9A3
:107E4000071E06D0002303712378012B08D0132BC3
:107E500023D0A868002800D178E003F045FC75E045
:107E60006288029909A800F0A6F80290380000F094
:107E70008BF909AA2378387A019200223100009206
:107E8000029A00F012F9380000F064F9029B002B0E
:107E9000DFD0300000F080F9DBE70378032BD8D186
:107EA0006288029909A800F0D6F8DEE7122B13D1F8
:107EB000029909A800F0B5F8021EEAD127498B887B
:107EC000002BC6D0887909A92378019161780091A7
:107ED000310000F0EAF8BCE7002302AA93833000E7
:107EE000617809AAFFF72AFFB3E71D4B0993F6E76C
:107EF000042B02D09A1F012AABD8184A043B9B00DE
:107F0000995A0029A5D0D218907831003A0000F093
:107F1000AEF800289DD13B88042B03D0012130000E
:107F2000FFF724FF012C04D1A868002801D003F03A
:107F3000DBFB280003F0D8FA8020039B00024340BB
:107F400018000DB0F0BD012800D182E701213000FA
:107F5000FFF70CFFEDE7C0463465FF1F2465FF1FE8
:107F6000010017000B7803704B784370CB788A7848
:107F70001B021343438070470A88030002700A887B
:107F8000120A42700A88012A06D14A8882704A88F9
:107F9000120AC2700420704702208242FBD14A8834
:107FA00004309A704A88120ADA708A881A718A88AC
:107FB000120A5A71EFE710B50400012082420CD971
:107FC0004B780A781B0213432380834206D1CB7877
:107FD0008A781B0213436380002010BD022BFBD163
:107FE000CB788A781B02134363804B790A791B0292
:107FF0001343A380F0E70B8803700B881B0A4370C0
:108000004B8883704B881B0AC3708B8803718B88E5
:108010001B0A4371CB888371CB881B0AC37108206C
:10802000704703000120082A14D14A780878120208
:1080300002431A80CA788878120202435A804A7929
:108040000879120202439A80CA798879120202439F
:108050000020DA80704710B504000120022A05D103
:1080600000204B780A781B021343238010BDF8B51B
:10807000060010200F00150003F03EFC0400012054
:10808000002C0ED0A0230C22290023806780201D05
:10809000002D07D003F098FA2100300003F06CFAAD
:1080A0000020F8BD03F020FCF6E7F7B51E000090B5
:1080B00008AB142017001D78019103F01DFC041E6D
:1080C00012D0A2230370019B47704380099B057166
:1080D00046710C220830002B07D0190003F074FA07
:1080E0002100009803F048FAF7BD099903F0FCFB62
:1080F000F6E737B5041E0FD04388002B0CD00025BF
:10810000C1881323007A172201950095FFF7CDFF50
:10811000FF2365806372257037BD000010B50C49E0
:1081200004004A88002A09D08B89002B05D0002042
:10813000CB8A0222834201D010BD012213000A2003
:10814000434300204032C854C81842800472F3E709
:108150000665FF1F0023438003707047094B002111
:108160001A0010B55C88002C06D01C79844203D11B
:108170000A234B43D01810BD01310A330329F1D132
:108180000020F8E70665FF1F10B50400407A03F0F1
:10819000A3F9FF23637210BD7047043010B580B29D
:1081A00003F0EAFA002803D00421494203F014FA4C
:1081B00010BD000070B50025104CA0682580A58179
:1081C000A580A84202D003F08FFAA56000250C4CD0
:1081D0000C4B606D1D80230058331D70A84202D0E7
:1081E00003F082FA656500256068002801D003F07D
:1081F0007BFA013508340A2DF6D170BDCC65FF1F1E
:108200007065FF1FC065FF1F70B5041E09D1054DC5
:108210002880A881A880A868002802D003F064FA0A
:10822000AC6070BDCC65FF1FF0B54B8885B0019385
:10823000002343600A7905000F00022A00D07BE08A
:10824000CA88032A17D98B685E7819783602DC78D9
:10825000D8790E4399781B7A24021B020C430343FE
:1082600053495BBA0B80331D93421ED1042C04D0BA
:10827000631F022B0ED9012015E0019A4D4B12010C
:10828000D35A002B06D00198FFF7BEFF4A4A136964
:10829000013313610421B8682E812C80494203F018
:1082A0009BF96860002005B0F0BD434D042C06D05A
:1082B000631F022B0FD9EB680133EB60DBE7019AF8
:1082C0003C4B1201D35A002B05D00198FFF79CFFBD
:1082D0002B6901332B61374B30000293019B029ACB
:1082E0001B010193002301998C468B5213006344B8
:1082F0009C8003939E81FFF750FF039B041E9860B0
:1083000016D00421B868494203F066F9FA880100E2
:10831000043A200003F058F90199029AFB888A5A1E
:10832000043B9B18029A8B522B6801332B60A2E707
:10833000AB690133AB619EE71E4B0293019B1E01AB
:10834000029BF35A002B2DD002998C19A0680028AB
:1083500028D0012A26D1FA889B189BB27352A18992
:10836000994217D39B1AC018B96803F02DF9029BE4
:10837000A289F35A934200D07DE700222B81A38883
:108380002B80A3686B60029BF2520B4A5368013347
:10839000536070E7084A9368013393600198FFF7D0
:1083A00033FF68E7044A536901335361F6E7C04677
:1083B0003665FF1FCC65FF1F3C65FF1F70B5051EAE
:1083C00015D10B4C0B4B1880230058331870606D7F
:1083D000002802D003F088F96565250050356068F3
:1083E000002801D003F080F90834AC42F7D170BD09
:1083F0007065FF1FC065FF1FF0B51700A12285B093
:10840000920001934243394B06001B680C009B18F5
:10841000D933FF331D78FDF741FF0430854204DD79
:108420003000FDF73BFF0430C5B2BD4207D33A0030
:1084300000213000019B03F0DFF805B0F0BD2900FA
:10844000380002F0B1FF2300C6B250331E70039310
:10845000019B29006365380002F08EFFCBB20293C6
:10846000002B02D0039B01361E70002623005033E0
:1084700003931B78B34204D8606D002831D10020EB
:10848000DBE7029A2800002A04D0013B1000B34227
:1084900000D02800F700E719387002F0ADFF7860CF
:1084A00000280ED03A78019903F08EF8019A3B78B3
:1084B0000136D3180E4A0193D369F6B20133D36162
:1084C000D4E7039B18706065A74205D1084A1320C2
:1084D000D36A0133D362B0E7606803F005F908346A
:1084E000F2E703F001F900236365C8E73409FF1FD1
:1084F0003C65FF1FF7B50D0007000421686803F015
:108500006BF82B89040003702B891B0A43702B889E
:1085100083702B881B0AC3702E8902250436F6B29D
:10852000F42E15D81B4B9F4214D10C2003F0E4F914
:108530001135011E0CD0902303708E3B0371043B58
:108540004380154B8460C680187803F015F8002529
:108550002800FEBD5C237B43104AD3180093583398
:1085600001931B78002B0FD10300320038000099D3
:10857000FFF742FF019B05001B78002BE8D1380074
:10858000009903F099F8E3E7054A0725536A013398
:108590005362DDE7FEFF00003465FF1F7065FF1FBB
:1085A0003C65FF1FF0B587B0009017200F00160044
:1085B0000193FFF7F2FD1325041E19D00C98031E3A
:1085C00002D00199201D9847030AE370052302AAEF
:1085D000A0700430908127700098667003A9938082
:1085E0000494FFF787FF051E02D0200003F07CF8FB
:1085F000280007B0F0BD0000F0B587B01F000CAB3D
:108600001B780391059301210DAB06001C780492A1
:1086100000F0D6F81425002821D02000FFF77EFDB9
:108620000135041E1BD01149059B0A7803700132E5
:10863000D2B2131EC68001D101231A000B70227121
:108640003000049B03990097FFF7ACFF051E09D18A
:10865000230021000648074A093303F0B5F9280032
:1086600007B0F0BD002363802370F8E73865FF1F73
:10867000F380001130750000F8B505000E00064CBF
:10868000064F2368002B02D031002800984704349D
:10869000BC42F6D1F8BDC046DC65FF1FF065FF1F88
:1086A0000123064A5B425380002313715362044A3C
:1086B000136053609360D36013617047F065FF1FD0
:1086C000DC65FF1F0200002310B506499C00085915
:1086D000002801D1625010BD0133052BF6D11320C3
:1086E000F9E7C046DC65FF1F034A5388181A434266
:1086F0005841404210407047F065FF1FF0B585B00B
:1087000002930AAB1F780CAB1B88009008000E0088
:1087100001920393FFF7E8FF05001120002D1BD104
:108720000E48FFF7E1FF04001520002C14D00622AC
:108730000B99A771E01D02F047FF019B30002371E8
:10874000029B29006371009B66802370039B656216
:10875000E381FFF791FF280005B0F0BDFFFF0000A7
:1087600010B5FFF7C1FF04000220002C12D0608872
:108770000121FFF781FF606A002801D003F0ACF807
:1087800028220021200003F0AFF8012300205B42E3
:108790006380207110BD000030B5074A074C558832
:1087A000010013780020A54204D05B1A59424B41C6
:1087B0005842104030BDC046F065FF1FFFFF00006B
:1087C000084A10B501230C00904208D0FFF78CFF37
:1087D000031E04D0037923405A1E9341DBB21800D4
:1087E00010BDC046FEFF0000024B1879431E9841A1
:1087F000C0B27047F065FF1F70B504000D00160091
:10880000FFF772FF002804D10D4B9C4200D01430BA
:1088100070BD416A03790520002907D012221A4051
:10882000102A02D10520002EF2D10F20DB06EFD551
:10883000897E0C20A9428941494249420840E7E724
:10884000FEFF0000030010B5002800D110BD034852
:10885000034A41889142F9D09847F7E7F065FF1F36
:10886000FFFF0000002330B5C45CCD5C6C40D454E5
:108870000133102BF8D130BD0F23002210B5C45C9A
:1088800064002243CA54C25CD209013BF7D210BD36
:108890000200010010B52032103102F0CDFE10BDF3
:1088A000F0B58BB00390102005931700049102F0EF
:1088B000DBFE0090102002F0D7FE009B13240190F5
:1088C000002B05D000280CD11324009803F004F8E5
:1088D000019B002B02D0180002F0FEFF20000BB01D
:1088E000F0BD102002F0C0FE0600102002F0BCFE19
:1088F00013240500002E00D1AEE0002819D010226C
:10890000002102F0F1FF32002900039802F094FEEA
:10891000041E0ED133787F2B51D830000099FFF719
:10892000ABFF009B1B787F2B53D801990098FFF772
:10893000A3FF300002F0D0FF002D02D0280002F08B
:10894000CBFF002CC1D1102002F08EFE06001020BB
:1089500002F08AFE0290002E7CD0002878D03A00E7
:108960000F3223000125121105D00F333B4015B201
:108970005A4253411BB26A1E1201002B33D0049B92
:10898000D2B298180099029AFFF76CFF013D1022AD
:108990000021300002F0A8FFADB2049F2D017D1927
:1089A000AF4242D0002C33D0300002F095FF029B42
:1089B000002B00D189E7180002F08EFF85E729001F
:1089C0003000FFF759FF28002549009AFFF74AFFBA
:1089D000A7E729000098FFF74FFF28002049019AD8
:1089E000FFF740FFA5E70F210F4004998A18D9B27D
:1089F0008F4208D9D15C06A819540133102BF6D147
:108A0000029A0199C0E7791A48424141C901F2E747
:108A10003900300006AAFFF725FF3200039806A9A7
:108A200002F00AFE10370400BAE7002CBCD1300077
:108A3000029906AAFFF716FF320006A9039802F072
:108A4000FBFD082204003100059802F0BDFDABE7F4
:108A50001324A9E71324AAE7002800D06EE733E720
:108A600004BC0011F0B58BB00F0016000225009079
:108A700000283FD0002A3DD00B1DDBB21800029326
:108A800002F0F2FD1135041E34D0FDF747FD05005C
:108A90003A000099201D02F0D7FEEBB20393E37079
:108AA0002B0CDBB22F0A00936370FFB22B0E2370E6
:108AB000A7700193FDF72CFD1022010006A802F01B
:108AC000C3FE2100029A04AB06A8FFF7E9FE051ECB
:108AD0000DD1039B08223370009B04A9B370019B46
:108AE0007770F370301D02F0AFFEFDF71DFD200022
:108AF00002F0F2FE28000BB0F0BDF0B58FB00D0013
:108B0000149E039004920593002A03D102242000AE
:108B10000FB0F0BD002EF9D00398FFF7E5FD142447
:108B2000071EF4D07278337812021A43B3781B040C
:108B30001343F27812061A43036A0192934201D357
:108B40000133E3D1002D03D03B7901249B07DED50F
:108B50000822002106A802F0C7FE059B1324043357
:108B6000DBB21800029302F07FFD051ECFD0059AFC
:108B70000499043002F068FE04223100280002F05B
:108B800063FE3900102210310AA802F05DFE2900B0
:108B9000029A06AB0AA8FFF783FE041E0FD1082233
:108BA00006A908A802F050FE0822311D08A802F00C
:108BB0007BFD012807D101990398FDF7C9FC280026
:108BC00002F08AFEA3E70124F9E7000070B51C4C0F
:108BD00005002368181E10D0002D14D11A78002A21
:108BE0000CD1981C083202F0EFFC02F02DFC01358C
:108BF000002808D123681D70012070BD0A331800B9
:108C0000082202F0E1FC2368002BF5D0122002F0CC
:108C100073FE061E0DD0C12321680370457002311A
:108C20001022023002F0D0FC23683100587802F0A4
:108C3000A3FC206802F050FE00232360DCE7C0465E
:108C40001866FF1FF8B504002020FDF755FB0D4EF8
:108C5000A700BB590500002B0DD000280BD0D878F9
:108C6000FF2809D108492A000C55F3590748033356
:108C7000611802F0A9FEF8BD290002F0F5FD0028F8
:108C8000F0D1F8E73466FF1F1C66FF1F9D9E0011A0
:108C900070B5064D84006359002B05D0D87802F0DA
:108CA0001BFCFF226359DA7070BDC0463466FF1F9B
:108CB00070B506008CB00C0015000021302268460B
:108CC00002F012FE31001022684602F0BDFD1D20A8
:108CD00021000322684402F0B7FD6846FFF7D8FD83
:108CE0002D21040003222800694402F0ADFD20007C
:108CF0000CB070BDF0B50700160097B001931CAB27
:108D00001D7830221EAB00910AA800211C7802F0C9
:108D1000EBFD102239000AA802F096FD1022002176
:108D200002A802F0E1FD0722310002A802F08CFD4A
:108D3000072202AB9818631E9C41019902F084FD42
:108D400002AB9C732B005A1E934102AAD3730021DD
:108D5000102206A802F0C8FD06221D9907A802F0FD
:108D600073FD1A2002ABC01806221F9902F06CFD99
:108D7000102200990EA802F067FD102202AB0EA986
:108D800008781C78013A6040D2B208700133013192
:108D9000002AF5D10AA8FFF77BFD102212A90400D2
:108DA0000EA802F011FC102206AB0EA908781D785F
:108DB000013A6840D2B2087001330131002AF5D17E
:108DC0000AA8FFF765FD044310222098E4B212A917
:108DD00002F03AFD200017B0F0BD70B50E0014008F
:108DE0008CB00100102268461D0002F02DFD3100FC
:108DF000082204A802F028FD2100082206A802F09B
:108E000023FD6846FFF744FD04001022280008A94E
:108E100002F01AFD20000CB070BDF8B506000D0080
:108E200000243719AC4200D3F8BD02F025FC030A38
:108E30003B70631CDBB201379D4203D90234F0540E
:108E4000E4B2EEE71C00EDE773B506000C00022566
:108E5000002819D0002917D0032101A8FFF7DDFF52
:108E60006B469A793F231A40013313436A46300018
:108E7000937101A92200FFF71BFF051E04D10322F5
:108E8000E01C01A902F0A0FB280076BD037858077A
:108E9000DA08C00FD20080009B0710439B0F1843D5
:108EA000C0B2704707230B40C908C9000B430370C9
:108EB0007047000070B50400FFF7EAFE134DA400F0
:108EC0006359002B21D0186A002801D002F004FD5C
:108ED0002B59986E002801D002F0FEFC2B59D86E59
:108EE000002801D002F0F8FC2B59186F002801D09F
:108EF00002F0F2FC2B59586F002801D002F0ECFC74
:108F0000285902F0E9FC00232B5170BD3466FF1F85
:108F10000E4B8000C35870B50C00002B0FD09D681D
:108F2000002D0CD02B78201D0B706B784B70A97C1A
:108F3000FFF7B8FF2B7E23726B69E36070BD1022D0
:108F40000021200002F0D0FCF8E7C0463466FF1F85
:108F5000014B18607047C0463066FF1F074A030088
:108F60008000825810B5002A06D0D088984203D1DC
:108F7000012901D1FFF79EFF10BDC0463466FF1FD7
:108F8000F0B5264E95B087000B93BB5905000991AB
:108F900012200A92002B31D0D888FFF7A5FB0400DD
:108FA0001420002C2AD0280010A9FFF7B1FFBB59CC
:108FB0001E781D6A002E23D00895FDF7EFFA0700F2
:108FC0000020FDF7F1FA0790A379E61D069310AD96
:108FD0000CA9089800F0E2FA0EA9280000F0D7FAD0
:108FE0000B9B0A990493069B09980293079B03968F
:108FF000019300970EAB0CAAFFF77CFE15B0F0BDF5
:10900000FDF7CCFA06903000FDF7CEFAE31DA77904
:10901000079310AB06000893DAE7C0463466FF1FDB
:1090200030B50C4C85002A59030085B00120002A78
:109030000ED018006946FFF76BFF2B591A78D888B5
:10904000054B002A00D1054B6A46072100F0D9FBE9
:1090500005B030BD3466FF1F8F9500119D9500113E
:1090600030B5094C8500295985B010226846253154
:1090700002F0AAFA2A591121044BD0886A4600F05E
:10908000C0FB05B030BDC0463466FF1F39960011E5
:1090900030B5094C8500295985B010226846353114
:1090A00002F092FA2A591121044BD0886A4600F046
:1090B000A8FB05B030BDC0463466FF1F779600118F
:1090C000F7B54D4F86001020F4590D0002F0CCFA90
:1090D000F3592062186A132200286CD0033A290041
:1090E0009C6802F071FAF3591A780192002A58D15B
:1090F0001E6A227D317B944651400122019F11421C
:1091000001D167461740217D914339432175377B53
:109110004F40BC4660460027800701D44F081740E7
:10912000012102208F40227D82433A432275377B02
:109130005740BC4660460027400701D497080F40BF
:109140000420227DBF0082433A432275627D0027BE
:1091500094466046727B42400A4201D167460F4006
:109160000121627D8A433A436275777B5740BC4652
:1091700060460027800701D457080F400220627D17
:109180007F00824317436775767B00227E40760717
:1091900001D4BA080A400426617D9200B1430A4313
:1091A00062756A78002A08D06278002A05D0052204
:1091B0000533DA7700221000FEBD0422297911421E
:1091C00005D1A17C114202D10533033AF1E7019A9E
:1091D00021782C78002A02D10A00210014001822DC
:1091E0000429E8D8042CE6D805206043034A053357
:1091F0001218525CDDE7C0463466FF1F14BC001134
:1092000010B50A001121024B00F0FBFA10BDC04658
:10921000D39600110B0030B587B001AD2B806B46A3
:1092200004001100981D082202F0CEF92A000B213B
:109230002000024B00F0E5FA07B030BDFB960011AC
:1092400010B50A001121024B00F0DBFA10BDC04638
:109250004F97001113B50B0011006A4613706B464F
:1092600004000622581C02F0AFF96A4608212000CB
:10927000014B00F0C6FA13BD6F97001110B50A003C
:109280001121024B00F0BDFA10BDC046BF9700117E
:109290007FB505000B4BAA00D4580800002C0FD056
:1092A000666F237FE28821780396266F0296E66E2A
:1092B0000196A46E0094FDF709FC2800FFF7FAFD63
:1092C0007FBDC0463466FF1F10B51721FFF7E0FFD2
:1092D00010BD000070B50A000D00064B022104000D
:1092E00000F08FFA060029782000FFF7D1FF300048
:1092F00070BDC0469F96001170B586B000236A46C7
:109300001370836804001D78681E0A2859D801A9C3
:1093100002F06AFA060633373B3F43474B4F530090
:10932000180000F042F9062312284BD000281BD168
:109330006088FFF7D9F90823002813D04279002A62
:1093400047D1264B1A78072312070BD5244B1A68EE
:109350000723002A06D01668002E03D0290001AA90
:10936000B04703006A4613706B461B786088002B79
:109370002AD1FFF767FC06B070BD180000F06CF949
:10938000D4E7180000F087F9D0E7180000F093F94F
:10939000CCE7180000F0ADF9C8E7180000F0C3F9F9
:1093A000C4E7180000F0F6F9C0E7180000F0F6F97D
:1093B000BCE7180000F013FAB8E7180000F013FA41
:1093C000B4E707236A46137069466088FFF782FF97
:1093D000D1E70523012AC5D1024BB8E7C164FF1FBD
:1093E0002C66FF1F3066FF1FF8B52C4F8600F3591F
:1093F00004000D00002B40D0DA8882423DD15A781B
:10940000062A33D11A78002A2ED0012099681A6AC8
:10941000097D014206D0157B054203D007225A7010
:109420000120F8BD0220014204D0157B054201D085
:109430000922F4E70420014204D0127B024201D049
:109440000B22ECE7164B1B68002BE9D05B68002B66
:10945000E6D020009847BB5900215B78122BDFD162
:109460002000FFF715FFDBE70E4BECE7112A04D1D4
:10947000002900D032252900F2E7002D08D1200074
:10948000FFF732F9002803D0102302791343037148
:1094900021002800FDF798FAC2E7C0463466FF1F96
:1094A0002C66FF1F3066FF1F70B50E4E8500AB594E
:1094B0000400002B13D01B78002B11D10A4B1B6822
:1094C000002B04D05B68002B01D020009847735913
:1094D0005B78122B03D100212000FFF7D9FE70BD6D
:1094E000024BECE73466FF1F3066FF1F2C66FF1F40
:1094F000094B8000C3581020002B0CD01A6A002A98
:1095000009D09B68002B06D0127A1B7E101C9A4251
:1095100000D9181CC0B270473466FF1F70B5030035
:109520000D0014000220002A30D000292ED0137024
:109530000B78081D53704B789370FFF7A7FCE07011
:10954000012002212B7A23716B7B034063716A7BBC
:109550000A401343042263716E7B164033436371E8
:109560006E7BF608F600334363712B7B0340A371D7
:10957000287B014000200B43A371297B0A40134341
:10958000A3712A7BD208D2001343A37170BD10B51A
:109590000A0001000120FFF7C1FF10BD10B50A004D
:1095A00001000220FFF7BAFF10BD70B506000C00E5
:1095B0000220002E30D000292ED07378201D0B7091
:1095C000B3784B70F178FFF76DFC01223579257285
:1095D00071794B10080013409340104003438810EA
:1095E00010408000C9080343C9000B436373B1797D
:1095F0004B10080013409340104003438810024072
:109600009200C9081343C9000B4321202373FCF7C0
:1096100073FE854201D2122070BD2220257AFCF70C
:109620006BFE8542F7D823781820042BF4D8637892
:10963000012BF1D80020EFE7030010B5022000292C
:1096400009D0002B07D00322481C0A7019000D32E4
:1096500001F0BAFF002010BD03000222080010B57F
:10966000002B06D0002904D00E32591C01F0ACFFAB
:109670000022100010BD030010B50220002909D0FF
:10968000002B07D00422481C0A7019000C3201F08C
:109690009BFF002010BD10B5FFF7DEFF10BD0300DB
:1096A0000220002906D0002B04D0052200200A70D9
:1096B0001B784B70704703000220002B08D0002954
:1096C00006D05B7800200B70013B082B00D91830C6
:1096D0007047030010B50220002909D0002B07D0E5
:1096E0000622481C0A7019000A3201F06DFF0020A2
:1096F00010BD10B5FFF7B0FF10BD02000B00022037
:1097000010B500290ED0002A0CD00721197011883D
:1097100059701188090A997011180822D81C01F093
:1097200053FF002010BD03000A00022010B5002BDB
:109730000CD000290AD09978587809020143118089
:10974000901CD91C082201F03FFF002010BD03002F
:1097500010B50220002909D0002B07D00822481C90
:109760000A701900921801F02FFF002010BD0200AE
:109770000B00022010B500290BD0002A09D00921C6
:109780001970117818185970511C062201F01CFF2D
:10979000002010BD10B5FFF75FFF10BD02000B00E9
:1097A000022010B5002A09D0002907D0517819707D
:1097B00011180622581C01F007FF002010BD0300FD
:1097C00010B50220002909D0002B07D00A22481C1E
:1097D0000A701900063201F0F7FE002010BD10B526
:1097E000FFF73AFF10BD02000B00022010B5002A5F
:1097F00006D0002904D018005178FFF753FB002051
:1098000010BDF0B585B017001E006A46062305009E
:10981000080091819380FEF7C0FC1324011E029082
:109820000CD03800B047041E05D1280001A9FEF76E
:109830006FFA041E02D0029801F056FF2800FFF7CD
:1098400001FA200005B0F0BDF0B504008BB0019125
:1098500015000021102202A802F046F8334EA7009E
:10986000B85900283CD0C388A34239D10378002BD3
:1098700036D14278062A18D102000100553235311E
:109880000C3006ABFFF7A9FA002829D12000FFF71A
:109890002FFE020006A902A801F096FE200002A9F0
:1098A00002F042F801200BB0F0BD816E002917D004
:1098B0000B8A112A28D19D420ED101981231093A02
:1098C00001F0F2FE012807D1BB5920009D6EFFF781
:1098D0000FFE29000200DEE732212000FFF7D8FC4E
:1098E0002000FEF701FF061E1BD0416A002918D098
:1098F0000B8AAB4215D108220198123101F0D4FE37
:1099000001280ED1716A0AE09D42E9D1082201982E
:10991000123101F0C9FE0128E2D1BB59996E8A7E4D
:10992000B9E7200001F0A8FFBCE7C0463466FF1F7E
:10993000F0B56B4D87007E5985B033780290039364
:10994000002B00D087E0B368346A01937078062852
:1099500017D101221B7D134202D0217B114218D165
:109960000222134202D0217B114251D10422134220
:1099700003D0237B134200D08BE0019B5A7DEB592F
:1099800091E007380428F8D801F02EFF032E426733
:109990008300B36E002B03D11C2001F065FEB0667E
:1099A000EB599C6E002C1CD010220021200001F0ED
:1099B0009BFF0298FFF79CFD01002000FFF72DFAA6
:1099C00001F05AFE2082200008211230FFF725FA0C
:1099D0000298FFF78DFDA076EB592100D888FFF79C
:1099E0000FFC0822EB591CE0B36E002B05D01A00C7
:1099F000198AF0881232FFF70DFC0222019B197DB3
:109A0000EB5911423DD0207B10423AD0073208E09A
:109A1000F488FCF7DBFD01002000FFF711FC0A22AF
:109A2000EB595A70029B9C002A595378073B042B30
:109A300011D8D088FEF758FE00284ED0C3895A08A6
:109A4000D2182849029B0298CB542B594118043351
:109A5000254801F0B9FF05B0F0BDFCF79FFD0300FC
:109A60000120834201D100200393EB59DE88FCF7EB
:109A70009BFD039902003000FFF7ECFB019AEB59C4
:109A8000117D042211420CD0217B114209D00B22FE
:109A9000C7E7F688FCF73CFD01003000FFF7EEFB5E
:109AA0006BE7019A527D01210A4204D0607B084293
:109AB00001D00C22B5E702210A4204D0607B0842A3
:109AC00001D00E22ADE704210A4204D0627B0A4293
:109AD00001D01022A5E71222A3E7FA225200B0E734
:109AE0003466FF1F3866FF1FA79E001110B5064B96
:109AF0001A780423100018401A4200D00348FFF7D8
:109B000027FA002010BDC046C164FF1F7443FF1F29
:109B100070B50400FFF7D4FA051E43D12000FFF70B
:109B20007FFA234EA400A0598268937CDB0708D5F6
:109B30000321036A1B790B40012B02D1017F0B43E8
:109B40000377431DD97F8B1E022B0DD8022900D02D
:109B50000121C088FCF790FF042133591A7F597006
:109B60000A431A77280070BD01290CD10223102264
:109B7000437000210C3001F0B7FE30591021353010
:109B8000FFF74BF9EEE70529ECD10223D11843701A
:109B900010220C3001F018FD04233259117F0B43C1
:109BA0001377EAE708251828DCD1053DDAE7C04637
:109BB0003466FF1FF0B58BB0059143887E4F9E0041
:109BC000F45915000493002C15D1012902D000206E
:109BD0000BB0F0BD101D57781678FFF757F9EB68FA
:109BE000320002932B7A0499019300903B002000ED
:109BF000FCF70CFFEBE7E388049A934201D00820BE
:109C0000E6E72378012B00D1D4E0059B581E0928F4
:109C100000D9CFE001F0E8FD05CE0A29CC506C85D3
:109C20009AB229000498FFF773FFD1E720002900BA
:109C30001022453001F0C8FCB9594B78042B02D1F1
:109C4000013B4B70C3E70B000A00253335320C3162
:109C50000498FFF795F90498FFF702FA0522431ECE
:109C60009841BB59C0005A70B2E720002900102269
:109C7000553001F0A9FC049B4F4C9D0029590498D4
:109C80000A0006AB55320C31FFF77AF92959102238
:109C9000453106A801F008FD012808D10498FFF716
:109CA000F7F90590002804D106222B595A7005981F
:109CB0008EE708230593FAE763780C2B7AD1E36EDD
:109CC000002B03D11C2001F0CFFCE066BB59D86EFD
:109CD00000286FD01022290001F076FCBB590498AF
:109CE000DC6EFFF705FC0D22A076BB595A706EE7BB
:109CF000E06E00285ED063780D2B5BD12B880822A4
:109D00000382A91C123001F05FFCBB599A68517D97
:109D10000222114226D0186A407B104222D00C3217
:109D2000E4E763780E2B45D1236F002B03D1162077
:109D300001F09AFC2067BB59186F002803D010224D
:109D4000290001F041FC0F22BB59CFE763780F2BAC
:109D500030D1206F0622691C103001F035FCBB5950
:109D60009A68517D0422114203D0196A497B11423D
:109D7000D5D100210498FFF78BFA28E7636F002BF9
:109D80000DD0BB59586F0028F3D01022290001F0E4
:109D90001BFC0122BB5952425B6F1A61E9E7142098
:109DA00001F062FCBB5960675B6F002BE9D126E7CD
:109DB0002978DFE707200BE73466FF1F10B5064C54
:109DC000207001F0E1FC06212078FDF791FF0348A7
:109DD000FEF778FC10BDC0464766FF1F5D8F00117F
:109DE00000200BB270B50D00834216DA264B1878AE
:109DF00001F0C2FD041E0DD00378922B0ED0A02BD3
:109E000037D0224B1878FF283AD0210001F0B4FB5C
:109E1000002835D180200002684070BD43780E2BA9
:109E20000BD03E2BEDD18378052B12D0082BE8D137
:109E300081798088FFF7D8FA08E0154B82889A422A
:109E4000DFD183681878591CFEF7C0FE002817D1AF
:109E5000D7E7104B1B785B0712D50F4B1B68002B05
:109E60000ED09B68002B0BD0C289811D808898473B
:109E7000ECE7FFF741FAA068002801D001F034FCBC
:109E8000200001F031FBC5E74766FF1F6D43FF1F50
:109E900018200000C164FF1F3066FF1F10B5007856
:109EA000FFF712FA10BD10B50078FFF7FDFA10BDEC
:109EB0000C234343084A10B59B185A68002A03D064
:109EC000012901D1904710BD9B68002BFBD00029D0
:109ED000F9D19847F7E7C0466466FF1F0123834026
:109EE000094A10B5946B1C439463506B98435063BC
:109EF000D46B20009843012901D120001843D0637E
:109F0000116B0B43136310BD00800040F0B50024BB
:109F10000127154B85B0DA6B144E03921A6C01922F
:109F2000DA64019BE3403B4217D0039DE5403D408E
:109F30000295E5B202992800FFF7BAFF316A736A09
:109F4000002908D03900002B01D00299794028005F
:109F5000FFF7C4FF01E0002BF9D101340C36172CB8
:109F6000DFD105B0F0BDC046008000404866FF1F4D
:109F7000064B01215A68C2400A4204D01B68C34004
:109F80001800084070471B6DF9E7C046008000408C
:109F90000122064B8240002903D0D9680A43DA60C7
:109FA0007047D9689143D960FAE7C046003800404D
:109FB00030B5032444430F4BE25C1B199C785D7859
:109FC00001232D1B0135AB40013BA340A140DB43E6
:109FD0000C00122807D8084992005218116819403D
:109FE0002143116030BD054A11680B4023431360C3
:109FF000F8E7C0465BBC001108F0004014F00040D8
:10A00000C21F70B5D4B20623092C0BD80125084C09
:10A010009540002908D00021FFF7CAFF23682B4391
:10A0200023600023180070BD2368AB43F8E7C046E7
:10A0300000380040214BF0B51B185B78022B21D172
:10A04000032444431E4A1F4EA35C12199478012234
:10A0500015008540B76B013CE4B23D43A240B563B7
:10A06000194C122815D89B0000290CD117495B18F0
:10A0700099680A439A600123205C154A834011685D
:10A080000B431360F0BD11495B18996891439960C7
:10A09000F1E70E4B00290DD159690A435A61225C40
:10A0A0001328E8D00123203A93400A490868034363
:10A0B0000B60E7E7596991435961F0E74866FF1F74
:10A0C0005BBC001100800040A0BC001100F000400B
:10A0D000A0F00040A4F00040F8B500241B4E1C4D39
:10A0E0001C4B1B5D012B1FD1194A9269E2401A4299
:10A0F0000BD00122B25693402200143AD2B2022A67
:10A1000009D815494A6913434B61013402360C35AD
:10A11000172CE5D1F8BD0022B2560F499200521813
:10A1200091680B439360F0E7022BEED1E7B2380061
:10A13000FFF71EFF01235840C1B23800FFF77AFF36
:10A140003800FFF715FF6877DFE7C0462DBC001128
:10A150004866FF1F4966FF1F00F0004001220238D9
:10A160008240054B002903D059690A435A61704760
:10A17000596991435961FAE700380040F8B50E007B
:10A1800001210F008740114A0400D368FD43BB43FF
:10A19000D360831E8B4201D8FFF7E0FF002120002F
:10A1A000FFF72EFF0A4A0B4B5168012E05D13943A8
:10A1B0001B1951605E700020F8BD294051600222D9
:10A1C0001C1962709A6915409D61F4E700380040DF
:10A1D000008000404866FF1F012210B58240074BF7
:10A1E000002906D019680A431A600121FFF7C6FF4B
:10A1F00010BD196891431960F7E7C0460080004020
:10A200000C2370B5002543430A4A29009B181D7092
:10A21000094B04001B185D70FFF7B0FF0123A3403A
:10A22000064928000A681A430A6005490A689A43E1
:10A230000A6070BD6466FF1F4866FF1F34800040DF
:10A240003080004070B504000E00FF2813D00325B5
:10A250000540FFF7D5FF084AA3089B009B183F2243
:10A26000ED00AA40AE4019682000914331431960C7
:10A270000121FFF78DFE70BD18380040F8B50C24A1
:10A280004443134B0500E4186368002B03D1A36813
:10A290001220002B1AD0022201270E4B00215B193D
:10A2A0005A7028002770FFF769FF63681E1E08D0E8
:10A2B000A3683E00002B04D02800FFF759FE46405B
:10A2C000F6B228003100FFF709FE0020F8BDC046B5
:10A2D0006466FF1F4866FF1FF7B5C420FF222B4BA3
:10A2E00080001958002491433F3A0A431A508022B3
:10A2F000274F5202274E1A60274B1D5D002D21D09B
:10A30000A31E012B03D80121E0B2FFF727FF012D87
:10A3100018D11F4B9B69E3402B4213D0E3B21800C6
:10A320000193FFF725FE01000198FFF755FFE3B207
:10A33000143B022B1DD801217156184A8D405369D8
:10A34000AB4353613B7F002B0DD0E5B22800FFF7F4
:10A3500095FF2800FFF70CFE7B7F0100834202D0AF
:10A360002800FFF7A5FD01340C370236172CC3D1A6
:10A37000F7BD012100237156F3568D40074A9B001B
:10A380009B189A68AA439A60DCE7C04600E100E0A7
:10A390004866FF1F2DBC00114966FF1F00F00040FA
:10A3A00010B501210400FFF7E9FE0123044A002053
:10A3B00011194B70A34091690B43936110BDC046C6
:10A3C0004866FF1F70B50E0015000400FFF718FF68
:10A3D0000C236343094A20009B189D605E60FFF7D1
:10A3E0004DFFF021064B074A8900051E5A5002D046
:10A3F0002000FFF705FF280070BDC0466466FF1F00
:10A400000000FF1F0D9F001170B5134D07202C7821
:10A41000002C1FD1982221005200280000F0B4FF28
:10A420000123C420FF222B700C4B80001C635C6353
:10A430000B4B1C605C600B4B195891433F3A0A432D
:10A440001A50802252021A600D20074A074900F074
:10A45000BBFF200070BDC0464866FF1F0080004063
:10A46000A0F0004000E100E0D9A20011D9A0001145
:10A47000030010B50620072B09D8054A137001F018
:10A4800023F9D7210020034B034A89005A5010BDFD
:10A490009C43FF1F0000FF1FC91BFF1F70B51D005D
:10A4A00002240C2910D8094ACA40D2070CD5FBF760
:10A4B0002FFF041E08D1059A04992800FBF744FFDA
:10A4C000FCF7B2FDFFF712FB200070BD1210000078
:10A4D00030B50D7802232C009C43184201D02B4349
:10A4E0001C0008252300AB43284201D02B00234346
:10A4F00020241D00A543204201D01C4325002A230F
:10A500000D70184204D011781E3B0B43137030BD00
:10A510000028FCD10C2113788B43F7E7F8B51D0018
:10A5200006AB1B88140007AA0E000B201778002B1F
:10A5300027D10A78022A49D14A6850781178000256
:10A54000244A08438018042840D801F04DF903122A
:10A550001D1B2300F06800F0CFFF021CC0B2B84200
:10A5600000D93A1CD2B22000F1682A8001F02CF800
:10A5700006E00222F3681B882A8023701B0A63709E
:10A580000020F8BD0622EEE701232B80F3681B783C
:10A590002370F5E7F368002B16D008222A801A886A
:10A5A00022701A88120A62705A88A2705A88120A97
:10A5B000E2709A8822719A88120A6271DA88A2710E
:10A5C000DB881B0AE371DBE72B80D9E701202B80B6
:10A5D000D7E7C04600D6FFFFF7B516000A781D0082
:10A5E00008AB1F880C000123022A18D14A68507852
:10A5F000117800022B4A0843801803280FD801F075
:10A60000F3F802254439E06800F076FFC0B2072372
:10A61000B84204D37B190193152B02DD0D231800DA
:10A62000FEBDE0682A003100C01900F0CDFF6B4686
:10A6300000209B88E268D0541B4B1B68834203D0E8
:10A640001B68834200D098470023E8E70B23002FC4
:10A65000E5D1022DE2D1737832781B021343E26810
:10A660001380114B1B68002BEED01B68002BEBD026
:10A670000120E8E70B23002FD1D1062DCED12A00EF
:10A680003100E06800F0A0FFDEE70B23002FC6D109
:10A69000012DC3D132787533012AC0D8E3681A700E
:10A6A000D2E7C04600D6FFFF5468FF1F70B50C000C
:10A6B0001500072837D801F097F8041436361B36F2
:10A6C000242E182015290BD8184E162200213000F0
:10A6D00001F00AF922002900300000F075FF002087
:10A6E00070BD18200229FBD11288114B1A80F6E7A1
:10A6F00018200829F4D10A000E48290001F02CF98D
:10A70000EDE718200129EBD10B4B10780B49DA69E2
:10A71000FFF7DEFEE3E718200129E1D1064B1078B0
:10A720000749DA6BF4E70220DAE7C0463C68FF1F0E
:10A730001A44FF1F1044FF1FA043FF1FC843FF1F01
:10A74000E843FF1F030010B50020DB0704D50721F5
:10A75000024A034800F08CF810BDC046B8BC001196
:10A76000A043FF1F054A03001068002803D0828819
:10A770009A4201D1806870470068F6E74C6AFF1F73
:10A780000A88030008009A4204D08A8804309A425A
:10A7900000D0002070470000F8B5F22200230D4FD2
:10A7A0000D4E7968050042433370994200D07B60BA
:10A7B0000A4C0021200001F097F800231A007C6069
:10A7C000AB4202D100203370F8BD01332280DBB2EE
:10A7D000F234F5E7446BFF1F426BFF1F506AFF1F07
:10A7E00073B56B4601900600684615001980FCF7AA
:10A7F0004DFF041E11D1002D0FD07689002E11D0EF
:10A800000C2000F031FF00280ED0084A04601368C5
:10A8100086808560002B02D11060200076BD1A0072
:10A820001B68F7E70224F8E71324F6E74C6AFF1FDA
:10A83000012100220A4B10B549420A4C1980998027
:10A840009A719A70084B2070012019805A60FFF7A6
:10A85000A3FF2078FCF778FF0448FDF733FF10BD15
:10A860005C68FF1F4C6BFF1F446BFF1F1DA900118D
:10A87000022310B5002802D0FFF7B2FF0300180032
:10A8800010BD0000030010B50020DB0704D5042133
:10A89000024A0348FFF7A4FF10BDC046CCBC00111C
:10A8A0002044FF1FF0B50E2687B003930CAB1F8822
:10A8B00002ABF6180500080031000292FDF768F8B7
:10A8C00004000120002C0FD03088FFF74BFF03005D
:10A8D0000E20002B08D05E68002E05D02100280035
:10A8E000039B029A0097B04707B0F0BD0A4B10B522
:10A8F000984207D10122002352420A808B708A803D
:10A900008B7110BDFFF73CFF0028FAD001235B429A
:10A91000038000238370F4E7FFFF0000F8B5050013
:10A9200001290AD1134E00243388F227AB4219D0F3
:10A9300028001149FFF7DAFF06E0022904D10139A6
:10A94000FDF73EFF0028EDD0F8BD3B006343726881
:10A95000D018D35A002B09D03A00002100F0C4FFD0
:10A960000134E4B2054B1B78A342EED801235B42CD
:10A970003380DDE7446BFF1F5C68FF1F426BFF1FE6
:10A9800010B5FFF7FDFE03000020834200D0987849
:10A9900010BD0000F0B589B01C000EAB80CB039059
:10A9A0001E8810AB1B78049202930B7A0D00DB0615
:10A9B00016D42B780593022B24D00498FFF7D2FEEF
:10A9C000002812D003689C46002B0ED0029B220068
:10A9D000019329003B00644603980096A04705E0D8
:10A9E0000498FFF7BFFE002802D10E2009B0F0BD89
:10A9F0008368002BF9D00A22290003989847002881
:10AA0000D7D0F3E76B6858781A786B4B0002104385
:10AA10009842D2D8043B984210D2684B984242D018
:10AA200015D8674BC0180128C7D80B20002EDDD1E0
:10AA3000EB681A7859683A80200028E0614BC0180A
:10AA4000032800D979E000F0CFFE846A789E5E4B3F
:10AA50009842B2D10B20002EC8D101233B80EB6875
:10AA600031001B7823706889013080B2FCF790FFB9
:10AA70003A88031E0ED0017802328A183A80428941
:10AA800062704289120AA27059680278E01C00F0D4
:10AA90009BFD06E004323A8031000422601C00F085
:10AAA00023FF0020A2E70B20002E9FD1EB6807A90F
:10AAB0001E8804233B80330A300026706370FCF745
:10AAC00067FF051E28D004AB9A890E2304A95B18E2
:10AAD0003E49C668FCF7D0FF00280BD12B783C48D4
:10AAE0006A680599FBF786FB002803D1012304AAB5
:10AAF0005B42D3813278022A06D17168201D00F0B2
:10AB000063FD3B8802333B800E2304AA9B181B88FD
:10AB1000A3701B0AE370C4E704ABDE81F4E70B20EB
:10AB2000002E00D062E7E9680398FFF729FF0223AF
:10AB30003B802070000A6070B3E70B20002E00D02D
:10AB400054E70222EB681B883A8023701B0A63706B
:10AB5000A7E7E86800F0D0FCC2B203000720B242C9
:10AB600000D243E70DD00299DBB27118994202DBA3
:10AB7000921BD3B20293029BE9681A003B808919A9
:10AB80005AE70023F6E70B20002E00D02EE707221D
:10AB9000EB683A801A7822705A7862705A88A270EC
:10ABA0005A88120AE2701A792271DA886271DB8897
:10ABB0001B0AA37175E7C0460429000002280000A3
:10ABC00000D8FFFFFFD6FFFF03280000FFFF0000B3
:10ABD000FCBB0011F0B58DB06B460020089120221F
:10ABE0009B5E83423DDAA64B187800F0C5FE071E37
:10ABF00032D00378B02B2CD10079023816281FD818
:10AC000000F0CAFB17001E001E001E0031001E00CF
:10AC100096001E001D011E0052011E0073011E0041
:10AC2000CD011E0050021E001E001E008E021E00DE
:10AC3000E302944B94491B8878880B80FBF71AF841
:10AC40003800FCF79BFF914B1B68002B01D03800AC
:10AC50009847380000F048FC8020089B00024340E1
:10AC600018000DB0F0BDEE220021874800F03CFE38
:10AC70000BAA3B7B7989388900923A000D32FCF7A8
:10AC80009FFD0400804B1B78002C3FD146E0804B99
:10AC9000788805937F4B4100CB5A0BAE073BDBB264
:10ACA00032880293002301937B4B2100069300938B
:10ACB000059BFFF76FFE744D002810D1069B3A8A62
:10ACC0001B889A420BD138000599123000F0ECFC39
:10ACD000002804D02B7862899B00EB185A80162339
:10ACE00006A81B18328820007989FCF7C5FE2B784E
:10ACF00004009A00AA1851880029C3D00133DBB29E
:10AD00002B70002807D006A9C98A9180634A12884F
:10AD10009A42BCD802E0012149429180002B04D024
:10AD200059497888FAF7DAFF8AE73E890A2479E0F8
:10AD300000253E89574B06937B88069A5B009B5AF9
:10AD4000033B9D4202DB002DF0D05BE0162206A8FB
:10AD500012183B7B798900923A0030000D32FCF7E3
:10AD60002FFD0590002858D04689017A7888FCF795
:10AD7000F1FC041E44D1464B78880793069B4100A2
:10AD8000C95A454B0439C9B206AAD28A0693029120
:10AD9000019400930599079BFFF7FCFD041E2FD13A
:10ADA000069B39491A88931C002D26D14B8079883F
:10ADB000384B4900CB5A5119033B8B4220DD059B90
:10ADC00031485B8941190B71A91C0135C9B2EDB23B
:10ADD000059145191B0A2B71059B2D490433181841
:10ADE00000F0F2FB2C4B059A1B88D318DDB22C4BDC
:10ADF0009E4205D00136B6B29CE749889942D6D02A
:10AE0000002D0CD0204C2800618800F0FDFB207044
:10AE100021007888FAF772FF12E7059CF0E7002C12
:10AE200000D183E77B78142B00D109E716493B79E1
:10AE30004E800B700C717888FAF712FF00E7162429
:10AE400006ABE41821003889FCF7A2FD011E00D1F1
:10AE5000B7E1788822880F4C45002C5B0A4D013CF5
:10AE6000E4B2029400240F4B01940095FFF792FD89
:10AE7000041E00D014E129007888FAF74FFFDFE6BE
:10AE80004C6BFF1F0C43FF1F6468FF1F5868FF1FB8
:10AE90005869FF1F9464FF1F486AFF1F0A43FF1F82
:10AEA000FFFF00006668FF1F162406ABE4182100B0
:10AEB0003889FCF76DFD011E00D182E17888228877
:10AEC000AE4C45002C5BAE4D013CE4B202947C8953
:10AED000AC4B01940095FFF75DFD041E00D0DFE050
:10AEE00029007888FAF724FFAAE60025A44B1D80E4
:10AEF0003B00F6331B78A24A78880792AB4208D908
:10AF00009E4B12880693069943005B5A013B9A4276
:10AF100003DB0799FAF716FF92E616246B00FB187D
:10AF2000059306ABE418059B21001889FCF730FD5A
:10AF3000011E03D1059B01241E8973E77888924B7B
:10AF40002288069C099343001B5B904E013BDBB2B9
:10AF50000293002300960193099BFFF71BFD041E3B
:10AF600002D0059B1E895DE77B88069A5B009B5A91
:10AF7000079A108832881218934202DC1B1A013B90
:10AF800033807F4C023032880999001900F01CFB95
:10AF90002388328801359B182380EDB2A8E70BAADD
:10AFA0003B7B7989388900923A000D32FCF708FC26
:10AFB00000250590059B002B04D10A24002D00D10B
:10AFC0006EE060E0059B7888197AFCF7C3FB01000E
:10AFD000041E63D1694C6C4B788806940993069BD8
:10AFE0004400E45A694B063CE4B20BAE3288079346
:10AFF0000294019100930599099BFFF7CBFC041E75
:10B000004CD1079B5E491B881A1D002D30D14A8008
:10B01000059B5B4C5A8963191A716B1C9BB2E31830
:10B02000120A1A71162306A832881B187989059806
:10B03000FCF722FDFF21AA1C2E1D03350B000590F5
:10B0400092B2B6B2ADB2002803D006ABDB8AD9B259
:10B050001B0AA218651911712B714C4D301D2A88DD
:10B060004949201800F0B0FA2B88F618B5B2A1E7CC
:10B070004988914207D17A8806995200525AEB18B2
:10B08000053A9A42C4DC3E4C2800618800F08CF9F5
:10B09000207021007888FAF75FFED1E5002DF2D10B
:10B0A0003E89BFE6162606ABF61831003889FCF754
:10B0B0006FFC3D000400FA3500282DD0037A9B0672
:10B0C0000CD400227B893989788800923A000C32AE
:10B0D000FFF7E8FB041E10D03E8915E03088FFF72B
:10B0E00041FB00281AD08368002B17D021001222C0
:10B0F00078889847041EE4D0EEE72B78002B02D125
:10B100007888FAF739FE00262B78002B00D097E5D7
:10B11000002C00D194E585E60124DDE70E24DBE771
:10B12000162506ABED1829003889FCF731FC041E02
:10B1300047D0037A9B0611D4154A7B88118899421F
:10B1400003D01448814207D11380134BF2261D7897
:10B150000023D9B2A94221D30924A1E72888FFF707
:10B1600001FB00282FD08368002B2CD02100122255
:10B1700078889847041EDFD092E7C0469464FF1F8A
:10B180006468FF1F6668FF1F5869FF1F486AFF1F3A
:10B19000446BFF1FFFFF0000426BFF1F310059434C
:10B1A000546801336018615A0029D2D13C00083438
:10B1B0002100F22200F008FA21007888FAF7E4FD75
:10B1C0003EE501246CE70E246AE71D4B1A887B8854
:10B1D0009A4231D07888FAF7E1FD31E5F2230598FB
:10B1E00051684343CD18C95A00291FD03B7A012B1F
:10B1F0000BD16C88AB887888AA1D0094FFF752FBAE
:10B20000041E02D000233B722E88F2220021280067
:10B2100000F06AFB00232B80059B0133DBB2059312
:10B22000084B05991B78064A8B42D7D801235B420D
:10B230001380002CCED0F5E5002634000596EFE70C
:10B24000446BFF1F426BFF1F70B504000E0015001A
:10B25000FFF796FA031E08D131000548FFF790FA70
:10B2600003001120002B02D01C8000209D7070BDB7
:10B27000FFFF0000F8B50B4F06003B780D001400EF
:10B28000FF2B0ED00A2000F037FB011E09D0B1239E
:10B290000380002346800371C5800481387800F064
:10B2A0006BF9F8BD6144FF1FF7B50F0008A9060050
:10B2B000088809A90B240988002821D10234022B0F
:10B2C0001ED1557813782D021D432B008B4301931B
:10B2D0007334002B14D1FB68300019000093FFF782
:10B2E0004FFB019C85420BD02A0030000099FFF7EC
:10B2F000ABFF041E04D12A0030007989FFF7BAFFA2
:10B300002000FEBDF0B50E7885B003900AA8058830
:10B310000120022E0DD14C682778647824023C432A
:10B32000054FBC4205D10398DBB201960095FFF7AB
:10B33000BBFF05B0F0BDC04602290000034B10B5AD
:10B340001B68002B00D09847FEE7C046506BFF1FDC
:10B3500007B501A8FFF7F2FF044A05480021121AB9
:10B3600000F012F8F8F788FAFEE7C046546BFF1FAA
:10B370006444FF1F0000000001B40248844601BC81
:10B38000604700BF090E000001B40248844601BCBA
:10B39000604700BFB70E000001B40248844601BCFC
:10B3A000604700BF853BFF1F01B40248844601BCD3
:10B3B000604700BF090E000001B40248844601BC8A
:10B3C000604700BFC539FF1F01B40248844601BC75
:10B3D000604700BF4931FF1F01B40248844601BCE9
:10B3E000604700BF9137FF1F01B40248844601BC8B
:10B3F000604700BF4D39FF1F01B40248844601BCBD
:10B40000604700BF017F000001B40248844601BCD0
:10B41000604700BF8B52010001B40248844601BC62
:10B42000604700BF456B010001B40248844601BC7F
:10B43000604700BFB352010001B40248844601BC1A
:10B44000604700BFA930FF1F01B40248844601BC19
:10B45000604700BFD91B000001B40248844601BC0C
:10B46000604700BF5D3BFF1F01B40248844601BC3A
:10B47000604700BF5934FF1F01B40248844601BC35
:10B48000604700BFF30E000001B40248844601BCCF
:10B49000604700BF0D52010001B40248844601BC60
:10B4A000604700BFE932FF1F01B40248844601BC77
:10B4B000604700BFC9A9000001B40248844601BC2E
:10B4C000604700BFC521000001B40248844601BCAA
:10B4D000604700BF055E000001B40248844601BC1D
:10B4E000604700BF1147010001B40248844601BC17
:10B4F000604700BF434D010001B40248844601BCCF
:10B50000604700BFDD52010001B40248844601BC1F
:10B51000604700BF4550000001B40248844601BCAA
:10B52000604700BFDD66010001B40248844601BCEB
:10B53000604700BF056A000001B40248844601BCB0
:10B54000604700BF75A9000001B40248844601BCF1
:10B55000604700BF691F000001B40248844601BC77
:10B56000604700BF413BFF1F01B40248844601BC55
:10B57000604700BF8552010001B40248844601BC07
:10B58000604700BF594F010001B40248844601BC26
:10B59000604700BF3D18000001B40248844601BC6A
:10B5A000604700BF9136FF1F01B40248844601BCCA
:10B5B000604700BF2146010001B40248844601BC37
:10B5C000604700BF9D36FF1F01B40248844601BC9E
:10B5D000604700BFE94C010001B40248844601BC49
:10B5E000604700BF5549010001B40248844601BCD0
:10B5F000604700BF5522000001B40248844601BCE8
:10B60000604700BF0519FF1F01B40248844601BC12
:10B61000604700BF350E000001B40248844601BCFB
:10B62000604700BF5D17000001B40248844601BCBA
:10B63000604700BFC136FF1F01B40248844601BC09
:10B64000604700BFE548000001B40248844601BCE1
:10B65000604700BF2526000001B40248844601BCB3
:10B66000604700BF8539FF1F01B40248844601BC12
:10B67000604700BF3D4B010001B40248844601BC55
:10B68000604700BF2951010001B40248844601BC53
:10B69000604700BF5952010001B40248844601BC12
:10B6A000604700BF713AFF1F01B40248844601BCE5
:10B6B000604700BFCD4C010001B40248844601BC84
:10B6C000604700BF3119FF1F01B40248844601BC26
:10B6D000604700BFC91BFF1F01B40248844601BC7C
:10B6E000604700BFC56D010001B40248844601BC3B
:10B6F000604700BFD949010001B40248844601BC3B
:10B70000604700BF7918000001B40248844601BCBC
:10B71000604700BFB54C010001B40248844601BC3B
:10B72000604700BFC94A010001B40248844601BC19
:10B73000604700BFF919FF1F01B40248844601BCED
:10B74000604700BF851F000001B40248844601BC69
:10B75000604700BFA54F010001B40248844601BC08
:10B76000604700BFC130FF1F01B40248844601BCDE
:10B77000604700BF0124000001B40248844601BCB8
:10B78000604700BFE928000001B40248844601BCBC
:10B79000604700BFC926000001B40248844601BCCE
:10B7A000604700BF291C000001B40248844601BC68
:10B7B000604700BF4538FF1F01B40248844601BC02
:10B7C000604700BF6571010001B40248844601BCB6
:10B7D000604700BFED3AFF1F01B40248844601BC38
:10B7E000604700BFC51D000001B40248844601BC8B
:10B7F000604700BF713BFF1F01B40248844601BC93
:10B80000604700BF2124000001B40248844601BC07
:10B81000604700BF4D1F000001B40248844601BCD0
:10B82000604700BF3555000001B40248844601BCA2
:10B83000604700BF6DBC000001B40248844601BCF3
:10B84000604700BF9DA9000001B40248844601BCC6
:10B85000604700BF4551010001B40248844601BC65
:10B86000604700BF5125000001B40248844601BC76
:10B87000604700BF5147010001B40248844601BC43
:10B88000604700BF091B000001B40248844601BCA8
:10B89000604700BF156B010001B40248844601BC3B
:10B8A000604700BF193BFF1F01B40248844601BC3A
:10B8B000604700BFF94C010001B40248844601BC56
:10B8C000604700BF8D12000001B40248844601BCED
:10B8D000604700BFE117000001B40248844601BC84
:10B8E000604700BF014C010001B40248844601BC1E
:10B8F000604700BF154D010001B40248844601BCF9
:10B90000604700BF1D4D010001B40248844601BCE0
:10B91000604700BF2933FF1F01B40248844601BCC1
:10B92000604700BF692EFF1F01B40248844601BC76
:10B93000604700BF311B000001B40248844601BCCF
:10B94000604700BF1D4B010001B40248844601BCA2
:10B95000604700BFB14E000001B40248844601BCFC
:10B96000604700BF810E000001B40248844601BC5C
:10B97000604700BF053AFF1F01B40248844601BC7E
:10B98000604700BFF54E010001B40248844601BC87
:10B99000604700BFADAE000001B40248844601BC60
:10B9A000604700BFEDA5000001B40248844601BC19
:10B9B000604700BFED4A010001B40248844601BC63
:10B9C000604700BF3939FF1F01B40248844601BCFB
:08B9D000604700BFA946010019
:10B9D8000001010302030303040305020602070230
:10B9E800080209000A030B030C020D000E030F03E3
:10B9F800100311031303140315001600513C001122
:10BA0800853C001100000000020000001ABA001175
:10BA1800192A0F180A000000F1590000FD2400003F
:10BA280041460100CD7D0011E19D001135720011E4
:10BA3800D17B0011E1530011D5AB00113550001135
:10BA4800613E0011913F0011000000001616000031
:10BA58000200000064BA0011F4FFF3FFD2FC0000FA
:10BA6800D140001100000000000000005475796109
:10BA78000042322E30003030313400676974687506
:10BA8800622E636F6D2F707676780042544830319D
:10BA98000000000002000000B0BA0011292A282A7C
:10BAA800272A262A252A242A0A180000E204000048
:10BAB8007102000078EC00000500000074400000EE
:10BAC8001027000060F00000040000000664000079
:10BAD800204E000000000000060000005C4400004A
:10BAE800102700006CEE00000700000005000000B1
:10BAF8001F501D10023CB40000011400200000007B
:10BB0800810200003031323334353637383941421A
:10BB18004344454600000000E5570011395800111C
:10BB2800000000000200000038BB00116F2A6E2AD6
:10BB38001A18000001A00000000000006410B71DE2
:10BB4800C8206E3BAC30D9269041DC76F4516B6B43
:10BB58005861B24D3C7105502083B8ED44930FF005
:10BB6800E8A3D6D68CB361CBB0C2649BD4D2D386BB
:10BB780078E20AA01CF2BDBDFB349B5F8000008008
:10BB88000010000000000000375E0011C1740011B1
:10BB98005B5E0011C9780011DF5E00119F7800110B
:10BBA800555F001175780011A75F00113D7A0011EB
:10BBB8000F6000113D7A001141600011F779001102
:10BBC800555F00112D780011CD5F0011D579001156
:10BBD8000000000000000000B3600011D5790011DA
:10BBE80015610011D9740011052A042A012A002AB6
:10BBF8000229032801280028011800180000000065
:10BC080000000000000000000000008701010201A0
:10BC18000201010201020303040103010101010100
:10BC28000303020103000D000E00100011001300B1
:10BC38001401070108010A010B011C011D0204027D
:10BC480005020702080219021A021C021D03010359
:10BC5800020317000201000504000807000B0A0090
:10BC68001716001D1C010201010504010E0D01112A
:10BC780010011413011716011A19020201020B0A06
:10BC8800020E0D0211100214130217160305040305
:10BC98000807030B0A030E0D0001020307090A0B2C
:10BCA8000E0F101112141718191A1B1F2021220029
:10BCB8001DA50011D9A50011000000000200000018
:10BCC80002BC00110000000005B3001100000000D4
:08BCD8000200000000BC001195
:020000041FFFDC
:1000000000000000C93D001120BA00111CBA001107
:100010009461FF1F000000000000000000000000CD
:1000200000000000000000000000000000000000D0
:1000300000000000000000000000000000000000C0
:1000400000000000000000000000000000000000B0
:1000500000000000000000000000000000000000A0
:100060000000000000000000000000000000000090
:100070000000000000000000000000000000000080
:100080000000000000000000000000000000000070
:100090000000000000000000000000000000000060
:1000A0000000000000000000000000000000000050
:1000B0000000000000000000000000000000000040
:1000C0000000000000000000000000000000000030
:1000D0000000000000000000000000000000000020
:1000E0000000000000000000000000000000000010
:1000F0000000000000000000000000000000000000
:1001000000000000000000000000000000000000EF
:1001100000000000000000000000000000000000DF
:1001200000000000000000000000000000000000CF
:1001300000000000000000000000000000000000BF
:1001400000000000000000000000000000000000AF
:10015000000000000000000000000000000000009F
:10016000000000000000000000000000000000008F
:10017000000000000000000000000000000000007F
:10018000000000000000000000000000000000006F
:100190004D33FF1F9531FF1FC166010000000000B5
:1001A000000000000000000000000000000000004F
:1001B000000000000000000000000000000000003F
:1001C000000000000000000000000000000000002F
:1001D000000000000000000000000000000000001F
:1001E000000000000000000000000000000000000F
:1001F00000000000000000000000000000000000FF
:1002000000000000000000000000000000000000EE
:1002100000000000000000000000000000000000DE
:1002200000000000000000000000000000000000CE
:1002300000000000000000000000000000000000BE
:1002400000000000000000000000000000000000AE
:10025000000000000000000000000000000000009E
:10026000000000000000000000000000000000008E
:10027000000000000000000000000000000000007E
:10028000000000000000000000000000000000006E
:10029000000000000000000000000000000000005E
:1002A000000000000000000000000000000000004E
:1002B000000000000000000000000000000000003E
:1002C000000000000000000000000000000000002E
:1002D000000000000000000000000000000000001E
:1002E000000000000000000000000000000000000E
:1002F00000000000000000000000000000000000FE
:1003000000000000000000000000000000000000ED
:1003100000000000000000000000000000000000DD
:1003200000000000000000000000000000000000CD
:1003300000000000000000000000000000000000BD
:1003400000000000000000000000000000000000AD
:10035000000000000000000000000000000000009D
:10036000000000000000000000000000000000008D
:1003700051B3001100000000000000000000000068
:10038000000000000000000000000000000000006D
:10039000000000000000000000000000000000005D
:1003A000000000000000000000000000491BFF1FCB
:1003B000000000000000000000000000000000003D
:1003C000000000000000000000000000000000002D
:1003D000000000000000000000000000000000001D
:1003E000000000000000000000000000000000000D
:1003F00000000000000000000000000000000000FD
:08183800606FFF1F4118FF1F44
:10184000024981F3088802F0BFFB0000606FFF1FB0
:1018500070B500241E491F4A1F484C6308CA1B0567
:101860001B0DE4188242F9D11C4B80228B630021AE
:1018700009201B4B920519621A4B1B4DDA671B4B53
:10188000DA688243DA609A68194802409A60112047
:10189000296002F0B7F8112002F094F880226B6CF6
:1018A000112093436B64EE23DB006343114A1B0C4E
:1018B00013840122104B9A7201F022FC0F4B1B780B
:1018C000002B04D10E4B1021187802F015FB70BDCF
:1018D000000005408805054000060540FF010000A6
:1018E00000F0004004E100E0003800403CF000401F
:1018F000FFDFFFFF6461FF1F1862FF1F4664FF1FC9
:101900004462FF1F10B502F057FA072804D01228CE
:1019100008D0022808D010BD044A0420136B0133FC
:101920001363F8E70220F6E71420F4E73C65FF1F95
:10193000F8B507000C0026002500503630785135E8
:10194000002804D10300287058342370F8BD29788A
:10195000CA00481E8141A3183800A25C5B68C9B266
:10196000FFF7D0FF00280DD12B78DA00A218013341
:1019700050602B703378044A013B3370136A013393
:101980001362D8E70123DFE73C65FF1F5C23434375
:10199000074910B5C9180B0058331B78012B05D126
:1019A000FFF7C6FF034A936A0133936210BDC04636
:1019B0007065FF1F3C65FF1F10B502F03DFA064A37
:1019C0000121130010CB4942D967044B136002F088
:1019D0004BFB200010BDC04600E100E010001000ED
:1019E00010B5040002F028FA024B1C6002F03CFB28
:1019F00010BDC04600E100E010B5040002F01CFA82
:101A00004021094A200013688B43136000F0F6FA66
:101A100001F07EFC0022054B01201A60044B0432C9
:101A20001A6002F0A9F9FEE71CF00040C4F0004083
:101A3000C0F00040431E5A425341A022F0B5D201EB
:101A40005B421340154D164A40019B182A18127E1E
:101A50008BB00191002A1BD01A000832D46F0022EB
:101A6000E6B206AFE4B294420EDC2818C369002B3C
:101A700008D0019902AA117106AA049202AA16734B
:101A800003A898470BB0F0BD1978B9540132EAE7C2
:101A90001A7D1A7806AB01261A70E6E7FC67FF1F6D
:101AA00000400040F0B5254B04004001C25C85B009
:101AB000002A2BD01A18117E002927D0917E0029E8
:101AC00024D01179022921D11689D788D168F51B34
:101AD000ADB22A1C102D00D9102292B2BE4217D1ED
:101AE0001818012303710023C269C38003819A423D
:101AF00006D06846032103730171029301A8904741
:101B00000820002C00D0192001F0FAFA05B0F0BD31
:101B1000013C65426C41A0256442ED012C40084D1A
:101B20001B186419074D0633013A92B2AA42EDD050
:101B30001888461C1E80085C2070F5E7FC67FF1FB4
:101B400000400040FFFF00000F220E4B10B59868C8
:101B5000104002380A280BD802F00AF80D0A0B0AC6
:101B60000A110A0A0A0A060002210020FFF762FF92
:101B700010BD0121F9E70020FFF794FFF8E7DB6FC4
:101B8000F6E7C046004000400F220E4B10B59868A3
:101B9000104002380A280BD801F0EAFF0E0A0B0A9F
:101BA0000A120A0A0A0A060002210120FFF742FF70
:101BB00010BD01210800F9E70120FFF773FFF7E7E7
:101BC000DB6FF5E70090004013B5334C2378072B0B
:101BD0003DD8324B1A78324B002A39D1802219680D
:101BE00052020A431A60252001F0CCFE20232D4A20
:101BF00011680B43802113606B460422C9050868F5
:101C00000733104228D080210422C905C868104239
:101C10002ED080212020C905CA688243CA601422C0
:101C20001A701A78002A2FD18021C905C86820327D
:101C30000243CA6014221A701A78002A28D11A4B5B
:101C40001A7D22785A601D221A705932DA6013BD4B
:101C50001A6816490A40C5E7086802430A60142258
:101C60001A701A78002ACED01A78013AD2B2F7E761
:101C7000C8680243CA6014221A7019784A1ED2B288
:101C80001A700029F9D1C4E71A78013AD2B2C7E72D
:101C90001A78013AD2B2CEE79C43FF1F6444FF1F7B
:101CA0003CF000409443FF1F00200040FFFFFEFF78
:101CB000564B70B51B68012B03D1554A936D013308
:101CC000936501F0E9FF534B534A1860534B544C52
:101CD0001A600123534A1360534A13602378002B80
:101CE00006D006225149524801F066FF00232370B6
:101CF000504A514B10681B78C1B2002B0ED14F4C8B
:101D0000C0B223785BB2002B4FDB237824785BB220
:101D100064B21B0424021B191B1813600B1C5029EE
:101D20004ED95023464A47491078DBB2FF22022899
:101D30004BD10868444C454D267890432A7896420A
:101D400054D9227824782E78023B5D10A31B6B4374
:101D50005201D31A10335B111843086002F0ECF8FB
:101D6000031F012B45D83A4B1B78002B06D0394B6B
:101D70001B78002B02D0002001F09EFFA122364BE1
:101D800092009978354B4A431B689B188322920036
:101D90009B181B78033B012B03D8AF20400002F0B7
:101DA00013F801222E4BDA8270BD237824785BB2BF
:101DB00064B2FF33FF341B0424021B190138ABE764
:101DC000CAB2022AAED20223ACE70868254C264DDF
:101DD000267890432A78964208D9227824782D785C
:101DE000023B5B10641B63435201B2E72378DBB212
:101DF000B2E70228D5D11D4B1B78013B022B03D93A
:101E00001B4B1B78022BCCD16C20C8E79809FF1F15
:101E1000FC0FFF1F8864FF1FFF3F000014100340EA
:101E20008C64FF1F0C10034000100340D50BFF1FF4
:101E30007211FF1FB40003408C09FF1F680AFF1FC7
:101E4000490AFF1F94000340460AFF1F470AFF1F6D
:101E5000F908FF1F2209FF1F300DFF1F3409FF1F64
:101E6000BC0BFF1F440AFF1F450AFF1F1C09FF1F71
:101E70002309FF1F10B502F09FF80022014B1A80C2
:101E800010BDC0468464FF1F10B502F03DF8A121CB
:101E9000054A89009478054A61431268044B521838
:101EA000528C1A8010BDC046300DFF1F3409FF1F31
:101EB0008464FF1F10B50D4B0D4A9978A1239B0038
:101EC0004B431268D218531DD97F0A4B1B88994285
:101ED00009D2441C07D0C82805D0D2695B1A5A43DE
:101EE000054B5343C01802F057F810BD300DFF1FCB
:101EF0003409FF1F8464FF1F7102000070B5244D78
:101F00002B68002B28D001F04FFF2B68D8402B689E
:101F10000400002B27D001F0C7FE2B68D8401D4BD2
:101F20001D4A9978A1239B004B431268D118D25CBB
:101F300091239B00002A20D0CA580132CA50174B67
:101F400017491B680868834214D3D23B181A012A28
:101F50001AD0144B186070BD01F026FF124B19689F
:101F600002F052F8D3E701F09FFE0F4B196802F020
:101F70004BF8D4E70D495B18E8E7CA500C4B1B68D7
:101F8000DB68E418201AE4E7F530FF30E1E7C046EB
:101F90001C08FF1F300DFF1F3409FF1F9C09FF1F86
:101FA0008864FF1FA009FF1F1808FF1F2DFF3F00B7
:101FB0009064FF1F70B504000D00282916D103009E
:101FC000A433C2881B889B1A0B4A9BB293420DD93B
:101FD00006006A3605223100653001F085FF0028D1
:101FE00004D13100200001F03FFF70BD2900200026
:101FF00001F0F2FFF9E7C046FE7F0000F8B50500EA
:10200000012001F0B1FF134CA36AA26A9342FBD1F5
:10201000114E336001F068FE10490300086010485B
:10202000426894460F4A17680022BC4501D24268B4
:10203000BA1A0D4802603268AD18A422E562606ADF
:10204000520302436262094A1278002A01D00F3B10
:102050000B60F8BD00F00040340AFF1FE408FF1FCA
:1020600028100040180AFF1F1C0AFF1F1C09FF1F31
:1020700070B580241025E405A3682B43A36001F00C
:10208000B3FDA368AB43A36070BD0000F7B51600B5
:1020900080221C001023D2050191916805000B439A
:1020A000936000225A4BD7301A6001F0A5FE9D23A1
:1020B0002A002F009B00EB58CA3201210092FC3706
:1020C000002B01D00021009A386801F0C5FE2900DC
:1020D000009BCB311A784F4BD3351A604B780A7876
:1020E0001B0213438A7812041A43CB781B0613434E
:1020F000494A1BBA13604B790A791B0213438A7948
:1021000012041A43CB7931001B061343434A1BBA0E
:1021100013606B782A781B021343AA7812041A43BF
:10212000EB781B0613433E4A1BBA1360019A330235
:1021300013433C4A13603C4B22001B1B9C46032963
:102140003DDCB3089A0013005142B21A032A46D16B
:10215000354AE018511A827840781204000202438E
:10216000E05C043302430A600022FF2B4BDDF022C7
:102170002E4B12011A600F222D4B1A602D4A136844
:10218000002BFCD00023224A27491360091B321D73
:102190000B191B68043A180A23706070180C1B0E88
:1021A000A070E3700434002AF2DC802210213B6826
:1021B000D20501333B6093688B439360F7BD634660
:1021C000D578981893782D061B042B43157804397D
:1021D0002B43557804322D022B430360AFE7022ACC
:1021E0000AD1114AE05C511AE218527812020243F5
:1021F0000A6004339BB2B7E7012AB5D10A4A521AE2
:10220000E15C1160F5E7084959180A600433ACE74E
:10221000000004403C000440380004403400044006
:10222000300004400C00044000010440040004405D
:102230001000044014000440F7B5150080221C0073
:102240001023D2050091916807000B43936000238F
:10225000654AD730136001F0CFFD9D233E009B00FF
:10226000F9583B00CA363200FC33002900D07FE029
:10227000586801F0F1FD390032785C4BCB311A60BF
:102280004B780A781B0213438A78AC4612041A432F
:10229000CB78281D1B061343554A1BBA13604B7994
:1022A0000A791B0213438A7912041A43CB791B065D
:1022B0001343504A1BBA13604B7A0A7A1B0213432A
:1022C0008A7A12041A43CB7A21001B0613434A4A26
:1022D0001BBA1360009A2B021343484A1360220072
:1022E000474B1B1B0093009BCE785B1801938B78A8
:1022F00036061B0433430E78043833434E780431DA
:1023000036023343019E33600328ECDC0321A80826
:10231000431C9B002940800003292BD13849E51834
:102320005E18A9786D78E35C09042D0229431943EE
:102330003160030008330021FF2B2DDD314B324982
:1023400019600F21314B1960012327490B60304B75
:1023500019680029FCD006211B680B40042B20D0F3
:1023600080220020D20593680A318B439360FEBD22
:1023700001217DE7022908D121495D18E11849783A
:10238000E35C090219432960D3E70129D3D11C4931
:102390005918E35C0B60CCE7194818180160043346
:1023A000CAE7002310490B606346002B0CDC3B009E
:1023B000FC335A68102101325A608022D20593689A
:1023C00001208B439360D2E7009B9B181B68190A7E
:1023D00013705170190C1B0ED37004235B42917063
:1023E0009C440432E0E7C046000004403C00044046
:1023F0003800044034000440300004400C00044025
:102400000001044004000440080F000010000440D4
:102410001400044070B5061E19D002225A4B9B7955
:102420009343012B13D1594B1A78FF2A0FD15A78B5
:10243000FF2A0CD19A78FF2A09D1DA78FF2A06D12F
:102440001A79FF2A03D15B79FF2B00D199E0504B19
:102450000C201A78012A08D000224E4D1A702978D3
:102460000B00093B042B01D8212070BD4B1F012B11
:10247000FAD9454CA37B042B00D982E0A279032A28
:1024800000D97EE09A1ED2B2012A02D860881F28A5
:1024900077D9002E56D0012E73D1A0880128E3D021
:1024A000002907D1581E032803D801F061FB121739
:1024B00015122E702978481E032811D80025364B96
:1024C0001D602823237501F0DFFBA84227D0A580DB
:1024D000CAE702212970EDE70421FBE70321F9E7B0
:1024E00007390129C0D82D490968C96A8906BBD5B1
:1024F0002B4908780028B7D1012A01D9002BB3D184
:1025000002230B708021274D2633890128782375FB
:1025100001F002FD80212878890101F0EDFC012302
:10252000A380214B1B78002B0AD0FA2280211F4B5D
:1025300092001B8809025A431A4B187801F07CFB61
:10254000002092E701F078FC2B78A680073B012B56
:1025500003D917482E7001F0CFFB114B114C1A789C
:10256000002A06D080210022207889011A7001F00B
:10257000D3FC01F079FD80212078090201F0CCFC28
:10258000DEE7122071E7C046A60BFF1F6B09FF1F95
:102590001A09FF1F1C09FF1F4809FF1F9064FF1F36
:1025A0002309FF1F1B09FF1F2109FF1F2C09FF1F04
:1025B0000010004010B5002901D001F07DFC10BDD5
:1025C000F7B5604B01919978A1239B004B435E4A7C
:1025D000060014681022E418D6235B00E058362366
:1025E000FF33E35C00279343222B41D1574B0F3A33
:1025F0001A600760012501F0FFFC019B1880E823A9
:102600005B00E35C002B01D0B34258DD0023504F48
:10261000FB70AD33FF33E3581A68002A03D09B8860
:10262000DB439B071DD03823FF33E35C002B18D01E
:102630009B235B00E35C002B13D1D133FF33E35CBE
:10264000B3420EDAA4235B00E15AE018090A023112
:1026500001F0E2FB23000122FE33013E01351A871F
:10266000FA70E8235B00E35C002B2AD0A8B2FEBD21
:1026700003683D00002BBED081880430090A023176
:1026800001F0CAFBD6235B00E3581F60B2E72300CA
:10269000B133BA00FF339858013781880430090AF2
:1026A000023101F0B9FBE8235B00E35CBB42EEDCE6
:1026B000E822F61AED1800235200A354A6E70027DB
:1026C000F1E7200001F0C8FC00281FD0002E1DDD1E
:1026D0007319882647190193B600200001F02CFBDE
:1026E0005A30800020184068013581880430090A7A
:1026F000023101F091FB200001F04EFAA3590133A1
:10270000A351BD4202D0019B9D42E6D1114BE35C37
:10271000002BABD095239B00E35C002BA6D00E4B87
:10272000E15A0029A2D00D4AA35C994202D9013393
:10273000A3549BE700231A212000A35401F07CFC42
:1027400094E7C046300DFF1F3409FF1F00140340FB
:10275000E010FF1F5A020000720200005E0200003B
:102760000D4970B54A6E0D4CD2038B69D20BA24253
:1027700006D80B4D0224AA4204D901F045FA70BDD7
:1027800002246442E21815007E2425402242F4D03F
:10279000A3432B438B61F0E700F000400A200000C8
:1027A000FC1C0000F8B51D4B1D4F1A78002A10D1F3
:1027B000BA7B002A02D101321A7003E0032AFAD050
:1027C000022AF8D001F060FA00220120154B1A709D
:1027D000F8BD154B154D1C68154B9E7801232B70C9
:1027E0002878C0B200F09EFBBB7B002B0BD101F020
:1027F0000BFBA1239B007343E41883239B00E41885
:1028000023782B70E4E7032B02D101F065FBF0E79E
:102810000020022BDCD101F0D7F9EAE71C09FF1FE9
:10282000A60BFF1F2309FF1F3409FF1F490AFF1FC3
:10283000300DFF1FF0B587B00EAD2F780FAD2D789E
:102840000593AC46634614000E4D0CAA12782E7800
:1028500003930D9B009201932200059B029701F0C8
:102860007BFB2E70012C01D0042C08D1802206495C
:102870008B889343054A1278D20113438B8007B0AB
:10288000F0BDC0461C09FF1F6C11FF1F7809FF1F18
:102890000B001B3B70B504003020E02B0DD813005B
:1028A000E025493BFF3B9BB2ED00AB4205D8034B13
:1028B000200019825A8201F047FB70BD8410FF1F6F
:1028C00010B501F0E9F9054B00205B68052B04D930
:1028D000034A5268D20200D4980810BD001000408C
:1028E000FCE100E070B501F0A7FA0D4B1B68FC336A
:1028F000DC691D6AFFF7E4FF6419844204D2094BC6
:1029000001241B68002B07D004220024064B1A70F8
:10291000064A93690133936101F0A6FB200070BD64
:102920009064FF1F9809FF1F2309FF1FFC0FFF1F63
:1029300070B50C4D2B68FC335C6A01F07DFAFFF733
:10294000BFFF2B680025FC339B6AE318834204D247
:10295000054B1B68AB4200D1051B01F085FB28002D
:1029600070BDC0469064FF1F9809FF1FD722044B1B
:1029700092009B5810B5002B00D0984710BDC04660
:102980000000FF1F10B501F0DBF8FFF7EFFF27494C
:10299000274BCA6D274C1A4084235B001343CB6539
:1029A000254B1B68186A01F0DFFA244B244A1A6091
:1029B000244B254A1A60A022244B52001A60244B53
:1029C000187801F019F92000224901F02DFA0023AE
:1029D000A3600233A360204B2049236003232048D7
:1029E000A36001F021FA10221E4BFF201A60802202
:1029F00052031A60802292031A60802212041A6025
:102A000001F05AF9012001F087F9FA20400001F0A5
:102A1000B3FA582001F0D8F9134801F0DDF801208D
:102A200001F072F9072001F027FB10BD00F0004013
:102A300000FEFEFF141000409064FF1F00000340E2
:102A40000180063DBC00034034080000A4000340A0
:102A50004A0AFF1F71020000C3090000FFFF3F0088
:102A60002810004000E100E030750000674E336838
:102A700088331B6883F3088801F0CEF8644A6549FF
:102A8000136800200B401360634B644A1B68934239
:102A900000D1A6E001F0A0F90221614A13688B433E
:102AA0001360FFF76FFF5F4B5F4C1878C0B201F007
:102AB000EBF90023A3600233A3605C4B0120236089
:102AC00001F052FA0323A36001F02EFA040001F092
:102AD000E3F8050001F028FA554B186001F0B4FA4C
:102AE000544B1968621A531EA14200D2130080226F
:102AF000D203934201D39B029B0A3268D16AC90771
:102B000000D471E04C491C0C09689BB24C435943FA
:102B10002402090A641803264849FC3293680A68AB
:102B200047489B1A474A0768126847499B18474A13
:102B30009A1833409208DB190A600360042B03D90A
:102B4000013233400A6003600E684149A619300023
:102B500001F05AFA3F4F3E493B68C3183B603000D2
:102B6000019301F081F83C4E306808183849306014
:102B7000884205D9019B01333B6001F075F8316053
:102B800001F00AF9354B1B78002B0DD001F084F8C9
:102B9000334B621B196812188A4232D24919091B39
:102BA000091A304801F040F92F4E337A002B0ED02D
:102BB00001F072F8621BF1681218914224D9491988
:102BC000091B091A294801F02FF900233372284BF9
:102BD00083F3088801F078F8002001F0FDF800F098
:102BE000E3FF01F0F9F85CE7DC0199000234641AB4
:102BF0005900641A09214B438033CB40A408E418E0
:102C000089E7FA218900CCE71A49DBE79064FF1FC6
:102C10001CF00040FFFFC1FF0C0AFF1FB64121035B
:102C200010000040490AFF1F14100040C3090000B3
:102C3000100AFF1F340AFF1F380AFF1F200AFF1F58
:102C4000280AFF1F1C0AFF1F240AFF1FC4090000D7
:102C5000710200006008FF1F2C0AFF1F1C09FF1FE4
:102C6000E408FF1F00100040740BFF1F3C100040E1
:102C700000000020DC050000A022054B92009B58BC
:102C800010B5002B01D0984710BD01F005F9FBE706
:102C90000000FF1FA122054B92009B5810B5002B8E
:102CA00001D0984710BD01F0F7F8FBE70000FF1FC7
:102CB000A222054B92009B5810B5002B01D09847DB
:102CC00010BD01F0E9F8FBE70000FF1FA322054B50
:102CD00092009B5810B5002B01D0984710BD01F011
:102CE000DBF8FBE70000FF1FA422054B92009B5876
:102CF00010B5002B01D0984710BD01F0CDF8FBE7CF
:102D00000000FF1F70B500F0C7FF4F4B186001F0C7
:102D10004BF90400C30702D401F016F870BD00227D
:102D20004A4B1A604A4B18780138042829D800F019
:102D30001FFF0320181C2400200001F0C5F8012803
:102D4000ECD0444C2378042B6ED100F0C5FF002852
:102D5000E4D001F069F9582001F036F8022323701D
:102D6000DCE7200000F088FFE9E7200000F074FFB6
:102D7000E5E7200001F008F8E1E7200001F034F871
:102D8000DDE701F0D9F80500012808D1324B1B78A6
:102D9000053B012B03D82000FFF76EFFD1E72D4B39
:102DA0001B78022B01D0052B20D1022D28D12B4BD3
:102DB0009B7BAB431CD12000FFF76CFF264B1878A0
:102DC0000128BED16405BCD4244925224B7B034293
:102DD00005D1233A13405A42534126331A000B7D42
:102DE0009342AED9322001F047F8AAE7022D07D16D
:102DF000194B1B78052B11D12000FFF759FFDDE798
:102E0000012D0BD1012B03D12000FFF75FFF98E7C5
:102E1000062B03D12000FFF767FF92E7200001F0A7
:102E20003BF8022D8DD1C9E7032B04D10C4B987CC4
:102E300001F00AF872E7072B00D06FE7094B987B87
:102E400000F072FF6AE7C0469C09FF1F9809FF1F48
:102E50009009FF1F2309FF1F1C09FF1FA60BFF1F5F
:102E6000BC0BFF1FD40BFF1FFA210A4B0A4A490073
:102E70001A640A4A5A500A4A04395A50094A08310F
:102E80009A64094A5A50094A5C315A50084ADA662B
:102E90007047C0460000FF1F3528FF1F3129FF1F64
:102EA000E528FF1F1524FF1FA527FF1FB51EFF1FC5
:102EB000891EFF1FF7B50B0CFF270122009300238B
:102EC0003C001E001D009446019089B262469A4063
:102ED0001000084018413618B6B2FF2F02D1012E5B
:102EE00000D19FB2009802401A41AD18ADB2FF2C3C
:102EF00002D1012D00D19CB20133102BE6D1032069
:102F0000012E07D1012D04D1019B2401E4191C706D
:102F10000138FEBD102EFCD10238102DF9D0023040
:102F2000F7E700008023F7B59C46264B264F019318
:102F30002649274A274D284C284B02281AD160469B
:102F400038600868264E30408026360330430860DB
:102F500001990978002909D11660224A2A60224A7B
:102F60002260E02219689143A03A1BE08021C90247
:102F70001160F2E766463E600F68194E3E408027BA
:102F8000FF023E430E600199097800290DD11760B8
:102F900001280ED1154A2A60154A2260E0221968DC
:102FA0009143C03A0A431A60F7BD8021890211603B
:102FB000EEE7E0210F4A02432A600F4A22601A68B6
:102FC0008A43F0E74B0AFF1FE0000340D8000340AC
:102FD00090000340000003405000034040000340C5
:102FE000FFFFE3FF0280063D804508220180063D89
:102FF000806608220080069880550822F8B51E4B8E
:1030000080261A68002014003440324232D11A68F7
:103010001A4F32431A6001223B68063093433B60EB
:1030200000F0A2FF0122164D2B681E432E603B6864
:103030000A2613433B608027BF00124B1B683B42AC
:1030400011D1013EF6B2FF2E09D17E220E4B1C6833
:103050002B68E40B1440934323432B6005E00820C6
:1030600000F082FFE9E7002EEFD180222B68600894
:1030700093432B60F8BDC046C4F000405CF00040B4
:1030800018F0004068F0004060F0004010B501F01A
:1030900003F801215820034A00F0D6FDFFF7AEFFE8
:1030A00010BDC046600AFF1F10B5782200210348FA
:1030B00000F06AFF00F0F8FE002010BD8467FF1FDB
:1030C00070B5040000F0B8FE00230C200B4A01008C
:1030D00059438D18515C00290DD0A14208D101231C
:1030E00000246B7000F0A0FD00F0BEFF200070BD5A
:1030F00001330A2BEBD11224F6E7C0468467FF1F89
:1031000070B5040000F098FE002319001D000D4A60
:103110001078002806D0A0420CD1557001310C3235
:103120000A29F5D1002B0AD100F0BEFE00F09CFF69
:10313000002070BD5078461EB0411B18EEE700F02D
:1031400073FDF3E78467FF1FF7B504000C2000232D
:1031500084460E4D019267465F43E85D7E19A042AA
:1031600012D000280BD10A4B9C4662461B780833CC
:103170001370019B70707C557160B360FEBD0133AC
:103180000A2BE8D10320F9E70720F7E78467FF1F40
:103190008067FF1F8020F8B5484BC0051B68C1241D
:1031A0008360474BFF251A68012313434361454B56
:1031B000A4001A68444B40211A60444B1A68444BDF
:1031C0001A60444B1A59AA431A51C52292009E58BC
:1031D000AE433143802699509F583F49F6010F4036
:1031E0003E439E509E5880273602360A3043985000
:1031F00080201A5900020A4002431A5104341A5915
:10320000364E3F04324080263A431A511A59360648
:103210001202120A32431A5108341A5980260A40FF
:1032200002431A51C32292009F58B446AF4337431A
:103230009F509F58294E0F4007439F509F5837403B
:1032400080263604374380269F509F5836063F021B
:103250003F0A37439F50C0221F59AF433A431A5188
:103260001A591202120A1643C6221E5192009C5885
:10327000AC4365462C439C509C5800250C40204391
:103280009850C72080001A58154C1140C0221202D5
:103290000A431A50134B1B78DB08AB4201DC0020B9
:1032A000F8BD2378002B06D0A368002B00D09847E8
:1032B00001350C34EEE71220F2E7C0469843FF1FB9
:1032C0009443FF1FB0F000407C67FF1FB4F0004044
:1032D0007867FF1F00E100E0FF00FFFFFFFF00FF36
:1032E0008467FF1F8067FF1F030010B51F2809D8E0
:1032F000072200201340072404490A78A2431343FD
:103300000B7010BD00230620F5E7C0468067FF1F45
:10331000034A0449136800200B4013607047C046FD
:103320001CF00040FFFFC1FF054B06491B780A68EF
:1033300005485B0702401B0B134300200B607047DE
:103340008067FF1F1CF00040FFFFC1FF70B50C2518
:10335000FFF7EAFF0A4B1C780A4BE4086543ED18B7
:10336000002C01D1200070BD2B78002B06D06B689B
:10337000002B00D09847013C0C3DF1E71220F2E70A
:103380008067FF1F7867FF1F1FB5002102220B0017
:1033900001910091052000F077FE02230B490A6895
:1033A0001A42FCD120230393039B5A1E0392002B45
:1033B000FAD1074A1368002BFCDA0B246C44200076
:1033C000012100F029FE207804B010BD90C8004013
:1033D00000C8004013B504000A4B0193019B002B69
:1033E00001D1112016BDFFF7CFFF23000340044297
:1033F00005D0052000F0B8FD019B013BEDE718006A
:10340000F0E7C046FFFFFF0707B500F015FD80227B
:103410000821D205936A0191002B01D107399162ED
:1034200002210C4A11600199481E01900029FAD12D
:1034300003311160053101910199481E0190002965
:10344000FAD11160002B02D18022D205936200F0E4
:103450000BFE07BD00C00040F0B52D4C89B02378AD
:10346000002B4FD1FEF7A8FA02232A4F03903A68A7
:103470001A42FCD120230693069B5A1E0692002B6B
:10348000FAD1254E3368002BFCDA0120FFF7A2FFAA
:10349000011E02D0112009B0F0BD030003220190EB
:1034A000009005AD9F2000F0EFFD0321280000F003
:1034B000B3FD02233A681A42FCD120230793079BED
:1034C0005A1E0792002BFAD13368002BFCDA012038
:1034D000FFF780FF0028DDD10398FEF781FAAA7874
:1034E0006B7811041B020B4329780B4363601300B4
:1034F000113B0A49052B07D801239340A3600B60B9
:10350000012323700020C6E780231B03F6E7C04693
:103510008043FF1F90C8004000C800409808FF1F6C
:103520001E4B30B55A6818781D4B85B0D3185942D8
:103530004B4101210093002300F00EFC194B1A4A65
:1035400002259A6300221A6510325A658022C4212E
:103550009D65164B1648D202DA6789004258154B12
:1035600080241A4080231B041343435064234120CA
:103570000393E40500F006FA402000F003FA6562C8
:10358000039D6B1E0393002DFAD103236362FFF7A3
:103590003BFFA562FFF760FF05B030BD8C43FF1F06
:1035A00095FFFEF700C80040050001FF04E100E0C0
:1035B00000E100E0FFFF00FFF0B585B00700FEF777
:1035C000FBF9022305002D4C22681A42FCD120236E
:1035D0000093009B5A1E0092002BFAD1284E3368AC
:1035E000002BFCDA0120FFF7F5FE002803D01124A0
:1035F000200005B0F0BD234B2360022322681A424D
:10360000FCD120230193019B5A1E0192002BFAD179
:103610003368002BFCDA0120FFF7DCFE0028E6D13E
:10362000194B1F60022322681A42FCD12023029307
:10363000029B5A1E0292002BFAD13368002BFCDA4F
:103640000120FFF7C7FE0028D1D1104B23600223D1
:1036500022681A42FCD120230393039B5A1E039233
:10366000002BFAD13368002BFCDA0120FFF7B2FE01
:10367000041EBCD12800FEF7B3F9B9E790C800409A
:1036800000C8004001000006A8C8004001800001F9
:1036900010B50020FFF790FF10BD000010B5064BDD
:1036A00018705960FFF73CFF00211320034AFFF711
:1036B0004BFD002010BDC0468C43FF1F2135FF1F6E
:1036C000F0B5040085B003920291FEF775F98822E7
:1036D00063035B0B52051A438023DB059D6A80233D
:1036E000274F0092BA68002601901B039A420CD91A
:1036F000F82326001B041E401C4206D08022214BCA
:1037000052025E6219680A431A60002D0BD100F064
:1037100093FB02221C4B1A608023DB055A62013A9C
:103720009A6200F0A1FC0023039A934220D1002D5D
:103730000AD100F081FB144B03221D608023DB05BE
:103740005A629D6200F090FC8023BA681B039A4283
:1037500008D9002E06D000220A4B0C495A621A687A
:103760000A401A600198FEF73BF9002005B0F0BD51
:10377000009A0299D2181278CA540133D4E7C0468D
:103780008043FF1F00C8004000C00040FFFFFEFF55
:10379000F0B587B0029103920400FEF70DF9019095
:1037A00000F04AFB802302250122234EDB05356011
:1037B0005D629A6200F058FC204F3B682B42FCD1BE
:1037C00020230493049B5A1E0492002BFAD11C4D13
:1037D0002B68002BFCDA0120FFF7FCFD002802D04B
:1037E000112007B0F0BD2000039A029900F0BCFA46
:1037F000022304003A681A42FCD120230593059B5A
:103800005A1E0592002BFAD12B68002BFCDA0120FE
:10381000FFF7E0FD051EE3D100F00EFB802303223D
:10382000DB0535605A629D6200F01EFC0198FEF7D0
:10383000D7F8E0B2D5E7C04600C0004090C80040CD
:1038400000C80040F0B5802489B00600FEF7B4F847
:10385000E405A36A02250393029000F0EDFA012328
:10386000304F3D606562A36200F0FEFB2E4C236882
:103870002B42FCD120230593059B5A1E0592002B59
:10388000FAD12A4D2B68002BFCDA0120FFF7A2FDAC
:10389000002803D01124200009B0F0BD244B236080
:1038A000022322681A42FCD120230693069B5A1E4B
:1038B0000692002BFAD12B68002BFCDA0120FFF7CF
:1038C00089FD021EE6D11B4B03211E6003000190FF
:1038D0000090202000F0D8FB022322681A42FCD17D
:1038E00020230793079B5A1E0792002BFAD12B68BF
:1038F000002BFCDA0320FFF76DFD041ECAD100F097
:103900009BFA80230322DB053C605A629C6200F034
:10391000ABFB039B002B01D1FFF776FD0298FEF76E
:103920005FF8B8E700C0004090C8004000C8004001
:103930000100000694C8004007B50002019104226E
:10394000000A01A9FFF724FF0EBD000073B50500B2
:1039500005240B4AA3005B429B1819686B46DE1DC9
:103960003000FFF7A7FA022804D133782B55013C29
:10397000EFD276BD052CFCD00128FAD10230F8E751
:10398000140900111F2807D8012380228340D20583
:1039900091680B43936070473F2808D80123802229
:1039A00020388340D20551690B435361F3E75F2808
:1039B000F1D80123802240388340D205116A0B439D
:1039C0001362E8E71F2807D8012280218240C90539
:1039D0008B6893438B6070473F2808D80122802171
:1039E00020388240C9054B6993434B61F3E75F2858
:1039F000F1D80122802140388240C9050B6A9343E7
:103A00000B62E8E71F2810D880230200DB05153A77
:103A10001968012A06D820229143196019680A43BF
:103A20001A60704701228240F6E73F2811D88023B0
:103A30000200DB05353AD968032A06D810229143E3
:103A4000D960D9680A43DA60EBE701222038824066
:103A5000F5E75F28E5D842238022181A413B8340CE
:103A6000D205516A99435162516A0B435362D8E7B8
:103A700010B50400012813D1A022184992050B6843
:103A80005B015B0913430B60154B164A1968114023
:103A9000154A0A431A60402219680A431A6010BD89
:103AA0000028FCD101000A2000F09EFA21000B2022
:103AB00000F09AFAC0220A4B920019680A4340218A
:103AC0001A601A688A431A60B022044912060B6809
:103AD0005B015B0913430B60E1E7C04614F0004053
:103AE0001CF000407F00FEFF80FD010072B6074A17
:103AF0001368013313600422054B1A600023054A42
:103B000013608022D2055360FEE7C0467808FF1F8D
:103B1000C0F00040C4F0004005490B68002B05D1FF
:103B2000044A0A6004490A60044A13607047C046A8
:103B3000140AFF1F841E0000380AFF1FC4F0004053
:103B40000023034A1360034A1360034A136070475B
:103B500054F0004040F1004044F1004002B471468E
:103B600049084900095649008E4402BC7047C046C6
:103B700002B4714649084900095C49008E4402BC00
:103B80007047C04603B47146490840004900095ACD
:103B900049008E4403BC704701B40248844601BC0E
:103BA000604700BF5976010001B40248844601BC59
:103BB000604700BF8552010001B40248844601BC41
:103BC000604700BFE94C010001B40248844601BCD3
:103BD000604700BF19FA000001B40248844601BCE6
:103BE000604700BF8D11010001B40248844601BC4A
:103BF000604700BFDD3F000001B40248844601BCBD
:103C0000604700BFEDA5000001B40248844601BC36
:103C1000604700BFD1AE000001B40248844601BC39
:103C2000604700BFC9A9000001B40248844601BC36
:103C3000604700BF21A9000001B40248844601BCCE
:103C4000604700BF8B52010001B40248844601BCAA
:103C5000604700BF0167010001B40248844601BC0F
:103C6000604700BF0534010001B40248844601BC2E
:103C7000604700BF090E000001B40248844601BC41
:103C8000604700BF0934010001B40248844601BC0A
:103C9000604700BFA9D8000001B40248844601BCB7
:103CA000604700BFC95C010001B40248844601BC02
:103CB000604700BF6D0B010001B40248844601BC9F
:103CC000604700BFED6B010001B40248844601BCAF
:103CD000604700BF7997000001B40248844601BCE8
:103CE000604700BF01D7000001B40248844601BC10
:103CF000604700BFBD5C010001B40248844601BCBE
:103D0000604700BFC1A5000001B40248844601BC61
:103D1000604700BFE512010001B40248844601BCBF
:103D2000604700BF6911010001B40248844601BC2C
:103D3000604700BFC1F7000001B40248844601BCDF
:103D4000604700BFD9B0000001B40248844601BCFE
:103D5000604700BFDD0A010001B40248844601BC8F
:103D6000604700BFC56D010001B40248844601BC34
:103D7000604700BF9573010001B40248844601BC4E
:103D8000604700BFA1AF000001B40248844601BCF7
:103D9000604700BFF535010001B40248844601BC0C
:103DA000604700BFD544010001B40248844601BC0D
:103DB000604700BFE90B010001B40248844601BC22
:103DC000604700BFE927000001B40248844601BCF7
:103DD000604700BF7912010001B40248844601BC6B
:103DE000604700BF016C010001B40248844601BC79
:103DF000604700BFF935010001B40248844601BCA8
:103E0000604700BF8944000001B40248844601BCF9
:103E1000604700BFE9F6000001B40248844601BCD7
:103E2000604700BFC115010001B40248844601BCCF
:103E3000604700BF2D6C010001B40248844601BCFC
:103E4000604700BF75A9000001B40248844601BC68
:103E5000604700BF4DF9000001B40248844601BC30
:103E6000604700BF2144000001B40248844601BC01
:103E7000604700BF85C1000001B40248844601BC10
:103E8000604700BF6137010001B40248844601BCAD
:103E9000604700BF8914010001B40248844601BC98
:103EA000604700BFE917010001B40248844601BC25
:103EB000604700BFADAE000001B40248844601BCBB
:103EC000604700BFE9D4000001B40248844601BC49
:103ED000604700BF0134010001B40248844601BCC0
:103EE000604700BF75F8000001B40248844601BC79
:103EF000604700BFCD4C010001B40248844601BCBC
:103F0000604700BF0D52010001B40248844601BC65
:103F1000604700BFF9ED000001B40248844601BCCF
:103F2000604700BFB352010001B40248844601BC9F
:103F3000604700BF156B010001B40248844601BC14
:103F4000604700BFDD0C010001B40248844601BC9B
:103F5000604700BF116E000001B40248844601BCF6
:103F6000604700BF9D6A000001B40248844601BC5E
:103F7000604700BF0189000001B40248844601BCCB
:103F8000604700BF8512010001B40248844601BCAD
:103F9000604700BFB70E000001B40248844601BC70
:103FA000604700BF8937010001B40248844601BC64
:103FB000604700BFBD0B010001B40248844601BC4C
:103FC000604700BF8D82000001B40248844601BCF6
:103FD000604700BF59B3001101B40248844601BCD8
:103FE000604700BF51B8000001B40248844601BCDC
:103FF000604700BFB19F001101B40248844601BC74
:10400000604700BFCD0C010001B40248844601BCEA
:10401000604700BF090E000001B40248844601BC9D
:10402000604700BF3D71010001B40248844601BCF5
:10403000604700BF6DF6000001B40248844601BC31
:10404000604700BF53B9000001B40248844601BC78
:10405000604700BFC166010001B40248844601BC4C
:10406000604700BF71B0000001B40248844601BC43
:10407000604700BF9DA9000001B40248844601BC0E
:10408000604700BFF90D010001B40248844601BC3D
:10409000604700BF496D010001B40248844601BC7D
:0840A000604700BFED6801005C
:1040A80002000000FEBB00110100000010BA001160
:1040B80002000000FABB001101000000E840FF1FE9
:1040C8000200000018BA0011010000001462FF1F6E
:1040D80002000000F8BB0011030000008861FF1F08
:1040E8001200000002000000FEBB001101000000E9
:1040F80058BA001102000000FABB001101000000CC
:1041080055BA00110200000062BA00110300000055
:10411800C361FF1F02000000F8BB0011030000008C
:10412800D861FF1F02000000FABB00110100000067
:1041380054BA00110200000060BA00110300000028
:104148009961FF1F02000000F8BB00110300000086
:10415800BA61FF1F02000000FEBB00110100000051
:104168009CBA001102000000FABB00110100000017
:104178003142FF1F02000000AEBA0011010000002A
:1041880093BA001102000000FABB00110100000000
:104198003042FF1F02000000ACBA0011010000000D
:1041A800E061FF1F02000000FABB001101000000DF
:1041B8002F42FF1F02000000AABA001101000000F0
:1041C80083BA001102000000FABB001101000000D0
:1041D8002E42FF1F02000000A8BA001101000000D3
:1041E8007EBA001102000000FABB001101000000B5
:1041F8002D42FF1F02000000A6BA001101000000B6
:1042080079BA001102000000FABB00110100000099
:104218002C42FF1F02000000A4BA00110100000098
:1042280074BA00110202020202020000000000003B
:10423800161500004D4C0011114C00110CBB00115B
:1042480090011D0018001800FFFF07010203040574
:104258000602010600000000000000000000000047
:104268000000000000000000000000000000000046
:104278000300000002000000FEBB00110100000066
:104288002CBB001102000000FABB00110100000065
:10429800EC42FF1F0200000036BB001101000000C5
:1042A8000E62FF1F02000000F8BB001103000000AF
:1042B8007864FF1F02000000FABB00110100000033
:1042C800EC42FF1F0200000034BB00110100000097
:1042D8001062FF1F02000000F8BB0011030000007D
:1042E8007064FF1F120000000001000000000111AF
:1042F800FFFF000050485936000000000000000091
:104308000B000500F0000000B40000280028002879
:104318003075A000A000A000A00000080008E0017F
:10432800F0001000100010001000100010005000E5
:104338005000500010001000D007000000000000DE
:104348000F0001000500307507001000010081FF13
:1043580000000000FF00000099710011A16F00111A
:10436800316D0011FFFF0100FF000000B59B001137
:104378003199001149980011000000000000000068
:1043880000000800040000003B0001085902E00199
:1043980088212800FF00000002000000FEBB001179
:1043A80001000000C4BC001102000000FABB0011AB
:1043B800010000001D44FF1F02000000F6BB0011B1
:1043C800010000003C68FF1F02000000FABB00115A
:1043D800010000001C44FF1F02000000F4BB001194
:1043E800010000001A44FF1F02000000FABB001180
:1043F800010000001844FF1F02000000F2BB00117A
:10440800010000001044FF1F180018001D00900153
:10441800020000030202000002000000FEBB0011BF
:1044280001000000D8BC001102000000FABB001116
:10443800010000006044FF1F02000000F0BB0011F3
:10444800000000000000000002000000F8BB00119E
:0A445800030000005C68FF1F20FF56
:040000051FFF184180
:00000001FF
